:020000020000FC
:100000000240AC9000000000000000000000000072
:0200000280007C
:10000000FA088C982A310D00FA082A982A310D0036
:10001000FA083098013E003EFA083C98D180E6CFBD
:100020005B00DB00FB880000FA0848982A310D00CD
:100030002A49534F203531392D3420285341452D3D
:100040004A3138353020565057290D00E6D7000088
:10005000DB000000000000000000000000000000C5
:10006000FA08788DFA08F696FA080697FA080C97B7
:1000700000000000FA08189700000000FA086892D3
:10008000FA08E897FA08EE97FA08AC90000000002A
:100090000000000000000000FA088A98000000003C
:1000A000FA0864980000000000000000FA08C87B0D
:1000B0000000000000000000FA089C97D190E618AC
:1000C0000000E61C0F27E6180000D190E61900009A
:1000D000E61D0F27E6198813E6980004E69900004C
:1000E000E6980000DB009A9801C0CE989A9801D05B
:1000F000DE98DB0000000000FA081E9800000000F7
:10010000FA0846670000000000000000FA0824001A
:100110002A310D002A49534F203531392D342028FA
:100120005341452D4A313835302050574D290D0067
:100130002A49534F2032373134352D34202843415A
:100140004E2032392D353030290D002A49534F20A9
:1001500032373134352D34202843414E2032392D69
:10016000323530290D002A49534F2032373134358A
:100170002D34202843414E2031312D353030290D8A
:10018000002A49534F2032373134352D342028434B
:10019000414E2031312D323530290D002A49534F3F
:1001A0002031353736352D34202843414E20323921
:1001B0002D353030290D002A49534F20313537363F
:1001C000352D34202843414E2032392D3235302907
:1001D0000D002A49534F2031353736352D3420282C
:1001E00043414E2031312D353030290D002A4953FD
:1001F0004F2031353736352D34202843414E2031BC
:10020000312D323530290D002A49534F20313432F7
:1002100033302D3420284B5732303030292046617E
:1002200073740D002A49534F2031343233302D344A
:1002300020284B57323030302920536C6F770D0017
:100240002A49534F20393134312D3220284341522D
:1002500042290D002A49534F2031343233302D3496
:1002600020284B5732303030290D002A5341452089
:100270004A313933392D32310D002A49534F20315B
:10028000353736352D34202843414E2032392D352F
:100290003030290D002A49534F2031353736352D5E
:1002A00034202843414E2032392D323530290D007B
:1002B0002A49534F2031353736352D3420284341D4
:1002C0004E2031312D353030290D002A49534F2031
:1002D00031353736352D34202843414E2031312DEC
:1002E000323530290D002A49534F203531392D340C
:1002F00020285341452D4A31383530205650572952
:100300000D002A49534F203531392D3420285341CF
:10031000452D4A313835302050574D290D002A4996
:10032000534F2031343233302D3420284B57323064
:100330003030290D002A49534F20393134312D32C4
:10034000202843415242290D0031343A35313A30A8
:1003500036004170722031342032303135002A426B
:100360006C7565746F6F74680D002A5553420D00EB
:100370002A4344500D002A4453383030450D002A9A
:100380005344500D002A4144503138360D002A455F
:10039000210D004572726F7221202843616E206E1C
:1003A0006F7420616464206D6F7265206461746194
:1003B000206C69737420706172616D65746572730D
:1003C0002C206D6178696D756D2069732031332E35
:1003D000290D002A31002A310D002A534145204AB7
:1003E000313933392D32310D0000D7404E00F3F84A
:1003F000850B3D0DD7404E00F3F8860B3D08E11804
:10040000F7F8A890D7404D00F78EAE3EDB00E14CE8
:10041000E10EF78EA8900D4AC0C8D7404E00F428D0
:10042000820B47F23000CD0F47F23900AD0CF1A23C
:1004300027FA3000C2F4A890D7404D00E4A4AE3EA5
:10044000258FA8900D3247F26100CD1247F2660069
:10045000AD0FD02406F40A0026F46100F1A8C2F41E
:10046000A890D7404D00E4A4AE3E258FA8900D1D66
:1004700047F24100CD1247F24600AD0FD02406F4FA
:100480000A0026F44100F1A8C2F4A890D7404D001C
:10049000E4A4AE3E258FA8900D08E11EE118F7F800
:1004A000A890D7404D00F78EAE3E09C2C0C4D740D9
:1004B0004E00F484820B2D0249E02DAEDB00ECFDF2
:1004C000ECFEECFFF0D82804E014F6F40C903FE8C2
:1004D0004EE85FE8DA08EA03E00ED7404E00F68EF9
:1004E0005000F68E3890F68E0A90F68E6290F68E58
:1004F0006490F68E6090F68E5690F78E7D90E00FA9
:10050000F04EC085D7404D00F4C5AE3E3D02498057
:100510002D0949C12D0747FC0B002D0447FC0C0099
:10052000EA30640747FC0B003D05E028DA086A0959
:10053000C08F0D12F04EC084D7404D00F484AE3E03
:1005400047F80C003D05E018DA086A09C08F0D0471
:10055000E008DA086A09C08FF04F2842EA207206E4
:100560002841EA2072060842EA305E07E004B840FB
:10057000E6F5FFFFA8405C14D7404E00C4540000CD
:10058000A840F0640861B86046F62800BDF3E6F4C0
:100590006800D7404E00F6F40000E6F46A00D74049
:1005A0004E00F6F40200E6F4F100D7404E00F6F4F7
:1005B0000400E014D7504E00F6F40600F68E080052
:1005C000E6F4C400D7404E00F6F40A00E6F8320024
:1005D000DA087476E019E058DA08F259E6F83C00D7
:1005E000DA08CE0EF2F40A9048413D32E6F8640093
:1005F000DA087476E019E058DA08F259E6F83C00B7
:10060000DA08CE0EF2F40A9048413D22E00FF78E50
:100610007D90E6F8F401DA087476E018DA086A09E1
:10062000C08FE019E058DA08F259DA08B012F2F493
:100630000A903D0EE6F85402E6F92000DA08A476A6
:10064000EE90E138F7F87D90DA085010EA00640780
:10065000F2F40A90EA306407E6F84002E6F9200076
:10066000DA08A476EE90E118F7F87D90DA08700CBD
:100670000D79E6F83C00DA087476E019E058DA08FB
:10068000F259DA08B012F2F40A902D11E6F81400CB
:10069000DA087476E019E058DA08F259DA08B0128C
:1006A000F2F40A9048413D03E00FF78E7D90F2F49A
:1006B0000A903D58D7404E00F2F4580046F44100ED
:1006C0002D29E6F86400DA087476E019E058DA08B3
:1006D000F259DA08B012D7404E00F2F4580046F44E
:1006E00041002D18E6F86400DA087476E019E05845
:1006F000DA08F259DA08B012D7404E00F2F4580086
:1007000046F441002D07E00FF78E7D90E014F6F4DB
:100710000A900D28F04D49803D07E6F85402E6F9AD
:100720002000DA08A4760D14F04D49813D1148F2FD
:100730003D07E6F82402E6F92000DA08A4760D0861
:1007400048F33D06E6F80802E6F92000DA08A47648
:10075000EE90E128F7F87D90DA0850100D03E00FD5
:10076000F78E7D90F04EC087D7404D00F4A7AE3E87
:100770003D0249802D0B49A22D0949A32D0749A40B
:100780002D0549A52D0347FA09003D7048F03D6E3F
:10079000F68E0A90DA08E016C4400200F2F40A90DD
:1007A0003D62D44002002D5FF3F87D9007F8F8FF1A
:1007B00047F808009D44C0845C1406F4C0079C04FC
:1007C0000D070D0D0D130D190D1F0D250D2B0D31E1
:1007D000E6F8ED01E6F92000DA08A4760D30E6F837
:1007E000D201E6F92000DA08A4760D29E6F8B7016F
:1007F000E6F92000DA08A4760D22E6F89C01E6F975
:100800002000DA08A4760D1BE6F88101E6F9200045
:10081000DA08A4760D14E6F86601E6F92000DA0895
:10082000A4760D0DE6F84B01E6F92000DA08A4766F
:100830000D06E6F83001E6F92000DA08A476EE901D
:10084000D440020046F40B003D07E6F9DF00D480F7
:100850000200DA0836230D0AE6F93300D4800200DC
:10086000DA0836230D03E00FF78E7D90F04EC08539
:10087000D7404D00F4C5AE3E3D0249802D0249C629
:100880003D2548F03D1CDA080A82D7404E00F2F4BC
:10089000580046F441002D03E014F6F40A90F2F4F7
:1008A0000A903D0DE04FE6F81401E6F92000DA0861
:1008B000A476EE90E148F7F87D90DA083215F2F46C
:1008C0000A9048413D03E00FF78E7D90F04EC084C2
:1008D000D7404D00F4A4AE3E3D03F04E49802D02BA
:1008E00049A73D0E48F03D0CDA08E670F2F40A9094
:1008F0003D02E06F0D05F68E0A90E00FF78E7D90B9
:10090000F04EC084D7404D00F484AE3E47F8080056
:100910003D0C48F03D0ADA086C31F2F40A903D02D1
:10092000E07F0D03E00FF78E7D9008E1F04E43F875
:10093000A8909D0648F03D048A400200EA000005A8
:10094000DA087264E6F81001E6F92000DA08A47605
:10095000E038DA0874763FE84EE85EE8F68E0C90F0
:100960000804FCFFFCFEFCFDDB00ECFDECFEECFFF4
:10097000F0D8E006E6F5FFFFF0465C14D7404E00E5
:10098000C454000086F62700BDF7E006E005F046F7
:100990005C14D7404E00C454360586F6F301BDF70B
:1009A000E6F4C200D7404E00F6F40000E6F433004F
:1009B000D7404E00F6F40200E6F4F100D7404E00B6
:1009C000F6F40400E014D7504E00F6F40600F6F4F6
:1009D0000800E6F4E801D7404E00F6F40A00DA0811
:1009E000F88CE018DA087476E00BE08AE009E6F8A3
:1009F0005A00DA08C27AE008DA086095E008DA08F6
:100A0000BC95E6F81300DA084A5AF04D49802D02E9
:100A100049823D2FF68E08900D073AE8E8669A4025
:100A20000300E108EA00680CE6F4FA0042F40890DA
:100A30009DF4F68E0890F68E2E90D7404E00F3FC73
:100A40000200E064D7001400B9C43AE8E866F2F4A2
:100A50002E9048419D07E6F4C80042F408908D02AC
:100A60009A40F300DA08985C9A400300E108EA0033
:100A7000680CF2F40A903D5AF04D49802D024982EB
:100A80003D55F68E0890F68E2E903AE8E866F2F420
:100A90002E9048429D05E6F45A0042F408909DF5D8
:100AA000E6F45A0042F40890ED06E014F6F40A90D9
:100AB000E108EA00680CE6F81900DA087476D74015
:100AC0004E00F2FF360566FFFF00D7404E00F2FEF3
:100AD000380566FEFF00E6F4FF00204EF1C8E06432
:100AE000D7001400B9C4DA08BE57DA08BE57F2F4CA
:100AF0000A9048413D03E108EA00680C46FF0800FF
:100B00003D0346FE08002D0646FF94003D0646FEC6
:100B100094003D03E118EA00680C46FE8F003D0397
:100B2000E128EA00680CE108EA00680CF04D498011
:100B30002D034981EA30660CF68E0A90E00BE08ABC
:100B4000E6F94000E028DA08C27AE028DA0874768C
:100B5000E7FCF000E064D7001400B9C4F68E0890FA
:100B6000F68E2E903AE8E866F2F42E9048419D0504
:100B7000E6F4D20042F408909DF5E00BE08AE0B97B
:100B8000E008DA08C27AE6F8F401DA085C8F3AE89D
:100B9000E866E7FCC100E064D7001400B9C4DA08D5
:100BA000BE57E6F4C100F6F45490E048DA087476D3
:100BB000D7404E00F3FC0200E064D7001400B9C433
:100BC000DA08BE57D7404E00F2F4020004F4549005
:100BD000E048DA087476D7404E00F3FC0400E06485
:100BE000D7001400B9C4DA08BE57D7404E00F2F45B
:100BF000040004F45490E048DA087476E7FC8100BD
:100C0000E064D7001400B9C4DA08BE57E6F48100E6
:100C100004F45490E048DA087476F2F4549066F4E0
:100C2000FF00F1C8E064D7001400B9C4DA08BE5769
:100C3000F68E0A90DA08B012F2F40A903D12D7400C
:100C40004E00F2F4580046F4C1002D07D7404E0084
:100C5000F2F45C0046F48F003D02E1380D05E10836
:100C60000D03E1080D01E108FCFFFCFEFCFDDB00CB
:100C7000ECFD5FE83AE8E866F2F53890F0855C282C
:100C800020855C3800855C1806F81900DA0874764F
:100C9000F2F460904841EA30C80D3AE8E866E0595D
:100CA000E018DA08F257E6F83C00DA08CE0EF2F463
:100CB0000A9048413D45248F3890F68E0A90E6F818
:100CC000C800DA087476E019E058DA08F259E6F854
:100CD0003C00DA08CE0EF2F40A9048413D0CE6F4EE
:100CE000FF00D7404E00F6F45200E014D7404E000B
:100CF000F6F450000D1BE6F81900DA087476E05996
:100D0000E018DA08F257E6F83C00DA08CE0EF2F402
:100D10000A9048413D0BE6F4FF00D7404E00F6F440
:100D20005200E014D7404E00F6F45000F2F4389030
:100D300048458D08E014F6F46290F6F40A900D022E
:100D4000F68E3890E01DE6F82A00DA0890763AE848
:100D5000E866F04D5C14D7404E00D444500046F491
:100D6000E7033D05E6F82600DA0890760D13F04D0E
:100D70005C14D7404E00D4845000DA089679E6F827
:100D80002000DA089076E005F04D5C14D7404E0064
:100D9000C454500008D1D7404E00F2F45000404DEA
:100DA0009DD6D7404E00F68E5000E01DE10AD74098
:100DB0004E00E4AD820B86FD2502BDF9F68E6090F3
:100DC000E0D8DA0890760D47F2F4649048413D0689
:100DD000E014F6F46290F68E64900D3DF2F42490E7
:100DE00048463D1DF68E2490D7404E00F3F8840B04
:100DF00047F830003D06E6F81001E6F92000DA0871
:100E0000A476D7404E00F3F8840B47F832003D2318
:100E1000E6F84002E6F92000DA08A4760D1CE01995
:100E2000E058DA08F259E6F83C00DA08CE0EF2F49F
:100E30000A9048413D03248F38900D02F68E389079
:100E4000F68E0A90F2F4389048458D05E014F6F4D9
:100E50006290F6F40A90F2F46290EA20740CF2F4D4
:100E60000A9048413D124FE85EE8E6F86400DA086F
:100E70005E76E6F82A00DA089076E6F82100DA08CD
:100E80009076E0D8DA0890761F40FCFDDB00F68E05
:100E90000090F68E0290F68E2E903AE8E866F2F414
:100EA0002E9048419D08E6F43700E00522F40090BA
:100EB00032F502909DF2E6F43700E00522F400904E
:100EC00032F50290ED02E118DB00E108DB00E016EC
:100ED000E102E104F68E0A90F68E2E90F68E0090D6
:100EE000F68E0290F78EA990F78EAA903AE8E866FF
:100EF000F2F42E9048419D08F048F058BCF522F4D9
:100F0000009032F502909DF2F048F058BCF522F4C2
:100F1000009032F50290ED03E014F6F40A90F076BA
:100F2000F2F40A90EA304E10D7404E00F2F5360542
:100F3000F0865C18D7504E00C4585000D44850007A
:100F4000F7F8AA903AE8E866DA088E0EF128F2F48B
:100F50000090F2F5029026F4150038508D324920A9
:100F60003D30F0875C18D7404E00D448500046F41E
:100F700048003D07D7404E00D448520046F46B006D
:100F80002D06F067F78EA990F78EAA900D1AF046FD
:100F90005C14D7404E00D4545000C2F4A990404590
:100FA0002D01E1140861E6F5E703F0465C14D74033
:100FB0004E00C4545000F0760871F78EA990F78E59
:100FC000AA9049203D150861D7404E00F2F536053C
:100FD000F0965C19D7404E00C4595000F3F8AA901F
:100FE00005F8A990D7404E00D4495000F7F8AA90D0
:100FF00046F6F401AD0249202DA749413D03E01416
:10100000F6F40A90F0575C15D7404E00D4455000D6
:1010100046F448003D07D7404E00D445520046F400
:101020006B002D04E014F6F40A900D0DF0465C14EC
:10103000D7404E00D4545000C2F4A99040452D032F
:10104000E014F6F40A90D7404E00F6F65000DB00AC
:10105000ECFD5FE8F68E38903AE8E866E0F8DA08EA
:101060007476F2F460904841EA3094113AE8E86608
:10107000E059E018DA08F257DA08B012F2F40A90F0
:1010800048413D44E6F89600DA087476248F38909B
:10109000F68E0A90E019E058DA08F259DA08B01230
:1010A000F2F40A9048413D0EE6F4FF00D7404E00AE
:1010B000F6F45200E014D7404E00F6F45000F68EDD
:1010C0000A900D1AE6F83200DA087476E059E01852
:1010D000DA08F257DA08B012F2F40A902D0DE6F4AD
:1010E000FF00D7404E00F6F45200E014D7404E0007
:1010F000F6F45000F68E0A90F2F4389048458D08C8
:10110000E014F6F46290F6F40A900D02F68E389030
:10111000E01DE6F82A00DA0890763AE8E866F04D35
:101120005C14D7404E00D444500046F4E7033D051C
:10113000E6F82600DA0890760D13F04D5C14D740DF
:101140004E00D4845000DA089679E6F82000DA08D8
:101150009076E005F04D5C14D7404E00C45450002A
:1011600008D1D7404E00F2F45000404D9DD6E01D0E
:10117000E10AD7404E00E4AD820B86FD2502BDF9A1
:10118000D7404E00F68E5000F68E6090E0D8DA0818
:1011900090760D6FF2F4649048413D14E059E018E8
:1011A000DA08F257E014F6F46290E6F82A00DA085A
:1011B0009076E018DA08BC76E0D8DA089076F68EF9
:1011C00064900D57F2F4249048463D1DF68E24900D
:1011D000D7404E00F3F8840B47F830003D06E6F8A0
:1011E0001001E6F92000DA08A476D7404E00F3F8A3
:1011F000840B47F832003D3DE6F85402E6F9200042
:10120000DA08A4760D36F68E08903AE8E866E0181B
:10121000DA085E76F2F460903D05E6F4190042F4D7
:1012200008909DF3E6F4190042F40890ED19E019D6
:10123000E058DA08F259DA08B012F2F40A9048419C
:101240003D0D248F3890E6F8F401DA087476E01941
:10125000E058DA08F259DA08B0120D02F68E38902A
:10126000F2F4389048458D05E014F6F46290F6F4F7
:101270000A90F2F462903D04F2F40A90EA205810C9
:10128000F2F40A9048413D124FE85EE8E6F8640047
:10129000DA085E76E6F82A00DA089076E6F82100A9
:1012A000DA089076E0D8DA0890761F40FCFDDB0083
:1012B000ECFDECFEECFF06F0F8FFE004B840E00DBA
:1012C000E00EC4400200E6FF3A00E4800400E4803F
:1012D0000600F68E0A90D7404E00F68E5000F78E2C
:1012E000A990F78EAA90F68E0090F68E0290F68E58
:1012F0002E903AE8E866F2F42E9048419D07F04FB0
:10130000E00522F4009032F502909DF3F04FE005E5
:1013100022F4009032F50290ED03E014F6F40A9006
:10132000F2F40A90EA30F414D44002004841CD0DA2
:1013300008D1E6F5E703F04D5C14D7404E00C454E5
:101340005000F78EA990F78EAA9008D1D7404E0092
:10135000F2F53605F04D5C14D7404E00C4545000F1
:10136000F3F8AA9005F8A990D7404E00F3F8360597
:10137000F7F8AA90D7404E00F2F4360566F43F0025
:10138000B840D7404E00F2F4360546F48000FD0325
:1013900046F489008D10F2F4AC90EA20EE14D740A8
:1013A0004E00F2F4360546F4C000EAF0EE1446F4BE
:1013B000C900EA90EE14DA08BE5708D1D7404E00B3
:1013C000F2F53605F04D5C14D7404E00C454500081
:1013D000F3F8AA9005F8A990D7404E00F3F8360527
:1013E000F7F8AA90D7404E00F2F4360546F4F10023
:1013F0002D04E024F6F40A900D7DDA08BE5708D1DA
:10140000D7404E00F2F53605F04D5C14D7404E0043
:10141000C4545000F3F8AA9005F8A990D7404E00A4
:10142000F3F83605F7F8AA90E00EDA08BE5708D1AF
:1014300008E1D7404E00F2F63605F04D5C14D74077
:101440004E00C4645000F3F8AA9005F8A990F18CFE
:10145000F7F8AA90F2F70A903D03A840404EDDE568
:10146000D44002000841C440020048713D04E044F9
:10147000F6F40A900D3FD7404E00F6FD5000F3F809
:10148000AA9043F8A9902D03E118E4800600F08D9E
:10149000208EF0985C19D7404E00D449520046F493
:1014A0007F003D16D7404E00D449560046F47800E0
:1014B0003D0FD7404E00D4495000E4800400E6FFC1
:1014C0008813F0D828D4D7404E00F6FD50000D12F6
:1014D00046FF3A002D0FD7404E00D4595000F480FB
:1014E0000400C08440453D06E6FF3A000D03E024B9
:1014F000F6F40A90F2F50A90EA20E61248513D0609
:10150000D44002004841CD02F68E0A90F2F40A90CF
:1015100048423D02DA08B012F480060049813D03DA
:10152000E014F6F40A9006F00800FCFFFCFEFCFD57
:10153000DB00ECFDF68E38905FE83AE8E866F2F4FE
:1015400060904841EA304E163AE8E866E018DA085A
:101550008083F2F40A903D05E019E6F86400DA08A9
:101560000085F2F40A9048413D2EF68E0A90248FB1
:101570003890E6F8C800DA087476E018DA08808354
:10158000F2F40A903D05E019E6F86400DA080085F7
:10159000F2F40A9048413D0DE6F4FF00D7404E00BA
:1015A000F6F45200E014D7404E00F6F45000F68EE8
:1015B0000A90F2F438904845FD08E014F6F4629081
:1015C000F6F40A900D02F68E3890E01DE6F82A0037
:1015D000DA0890763AE8E866F04D5C14D7404E00A1
:1015E000D444500046F4E7033D05E6F82600DA0847
:1015F00090760D13F04D5C14D7404E00D48450000B
:10160000DA089679E6F82000DA089076E005F04DE1
:101610005C14D7404E00C454500008D1D7404E004F
:10162000F2F45000404D9DD6D7404E00F68E50004B
:10163000E01DE10AD7404E00E4AD820B86FD250295
:10164000BDF9F68E6090E0D8DA0890760D2AF2F4B3
:10165000249048463D1DF68E2490D7404E00F3F866
:10166000840B47F830003D06E6F81001E6F920004B
:10167000DA08A476D7404E00F3F8840B47F832001E
:101680003D10E6F81401E6F92000DA08A4760D0909
:10169000F2F4649048413D05E014F6F46290F68E51
:1016A0006490F2F462903D04F2F40A90EA203A1554
:1016B000F2F40A9048413D124FE85EE8E6F8640013
:1016C000DA085E76E6F82A00DA089076E6F8210075
:1016D000DA089076E0D8DA0890761F40FCFDDB004F
:1016E000ECFDECFEECFF2806E01FE004B840E6F459
:1016F0001440E0260060E047E964086128713DFC81
:10170000E6F4E007D7404D00F6F49C36E6F4E10736
:10171000D7404D00F6F49E36E6F4E207D7404D0080
:10172000F6F4A036E6F4E307D7404D00F6F4A2360F
:10173000E6F4E407D7404D00F6F4A436E6F4E507F6
:10174000D7404D00F6F4A636E6F4E607D7404D0044
:10175000F6F4A836E6F4E707D7404D00F6F4AA36CB
:10176000F78EA090E00DE10AD7404D00E4AD92362F
:10177000809D8DFAE0EAE069E018DA082A5F0EE859
:10178000E0A8DA087476F68E0A90E00DE10AD740F8
:101790004D00E4ADA43E808D8DFAE00DE00EE00733
:1017A000F04E5C14E6F5C8001BD502F40EFED740DF
:1017B0004D00C474AC3686FE62008DF2808D8DEED5
:1017C000E6F96646E6FA0800D4800200DA087E648C
:1017D000F78EA390F78EA590F78EA490E004884032
:1017E0008840884088408840E00CE01BE02AE6F909
:1017F000DF00E0B8DA08FC8B06F00A00F68E0090F5
:10180000F68E02900D023AE8E866F2F60090F2F7E2
:101810000290F046F05726F419003850ED03F3F823
:10182000A5902DF126F619003870FD0EE118F7F895
:10183000A390E014D7400300F6F4002FE6F45555CA
:10184000D7400300F6F4102FF78EA290F68E00908A
:10185000F68E02903AE8E866F2F40090F2F5029013
:1018600026F4F40138509D06F3F8A2903D03F3F8F6
:10187000A3902DF0F3F8A39049813D02E05F0D3372
:10188000F3F8A29049813D2EE014F6F43890F6F476
:101890000A90F2F63890D7404D00F486A43E2D0F02
:1018A000F0465C2420465C3400465C34D7404D0052
:1018B000D444AE3646F441003D02F68E0A90248FA1
:1018C0003890F2F4389046F409008DE3F2F40A906F
:1018D00048413D02E02F0D07E0B4B840E188F7F839
:1018E0007D900D01E02FF04F4982EA305A1AE00D49
:1018F000E10AD7404D00E4ADA43E808D8DFAE00DA5
:10190000E00EE007F04E5C14E6F5C8001BD502F4CB
:101910000EFED7404D00C474AC3686FE62008DF2D8
:10192000808D8DEEF78EA390F78EA590E004884011
:101930008840884088408840E00CE01BE02AE6F9B7
:101940003300E6F81D00DA08FC8B06F00A00F68E7C
:101950000090F68E02900D023AE8E866F2F60090EA
:10196000F2F70290F046F05726F419003850ED03D4
:10197000F3F8A5902DF126F619003870FD0EE11848
:10198000F7F8A390E014D7400300F6F4002FE6F434
:101990005555D7400300F6F4102FF78EA290F68E1F
:1019A0000090F68E02903AE8E866F2F40090F2F5C4
:1019B000029026F4F40138509D06F3F8A2903D03FE
:1019C000F3F8A3902DF0F3FAA09049A0FD12E00DDA
:1019D000F7FAA1900D0AF09D0892D7404D00F48DC2
:1019E0009236C088DA08C08C08D1C2F5A090405D5C
:1019F000EDF2F3F8A29049813D2FE014F6F438900F
:101A0000F6F40A90F2F63890D7404D00F486A43EE2
:101A10002D0FF0465C2420465C3400465C34D740F1
:101A20004D00D444AE3646F441003D02F68E0A9095
:101A3000248F3890F2F4389046F409008DE3F2F4E4
:101A40000A9048413D02E03F0D08E6F41D00B84011
:101A5000E1A8F7F87D900D01E03FF04F4983EA30AF
:101A6000B61BE00DE10AD7404D00E4ADA43E808DE9
:101A70008DFAE00DE00EE007F04E5C14E6F5C800CC
:101A80001BD502F40EFED7404D00C474AC3686FE62
:101A900062008DF2808D8DEEE6F96646E6FA08006A
:101AA000D4800200DA087E64F78EA590F78EA490A9
:101AB000E0048840884088408840E6F41000884070
:101AC000E6FCF800E6FB2200E03AE6F9DF00E0B8C9
:101AD000DA08FC8B06F00A00F68E0090F68E029073
:101AE0000D023AE8E866F2F60090F2F70290F0464E
:101AF000F05726F419003850ED03F3F8A5902DF1B6
:101B000026F619003870FD0EE118F7F8A390E014DE
:101B1000D7400300F6F4002FE6F45555D7400300F4
:101B2000F6F4102FF78EA290F68E0090F68E0290AB
:101B30003AE8E866F2F40090F2F5029026F4F40137
:101B400038509D06F3F8A2903D03F3F8A3902DF0D2
:101B5000F3F8A29049813D2EE014F6F43890F6F4A3
:101B60000A90F2F63890D7404D00F486A43E2D0F2F
:101B7000F0465C2420465C3400465C34D7404D007F
:101B8000D444AE3646F462003D02F68E0A90248FAD
:101B90003890F2F4389046F409008DE3F2F40A909C
:101BA00048413D02E04F0D07E0B4B840E1C8F7F806
:101BB0007D900D01E04FF04F4984EA304A1DE00D61
:101BC000E10AD7404D00E4ADA43E808D8DFAE00DD2
:101BD000E00EE007F04E5C14E6F5C8001BD502F4F9
:101BE0000EFED7404D00C474AC3686FE62008DF206
:101BF000808D8DEEF78EA090E00DE10AD7404D006C
:101C0000E4AD9236809D8DFAF78EA390F78EA59065
:101C1000E0048840884088408840E6F4100088400E
:101C2000E6FCF800E6FB2200E03AE6F93300E6F8CD
:101C30001D00DA08FC8B06F00A00F68E0090F68E86
:101C400002900D023AE8E866F2F60090F2F7029090
:101C5000F046F05726F419003850ED03F3F8A5903C
:101C60002DF126F619003870FD0EE118F7F8A39053
:101C7000E014D7400300F6F4002FE6F45555D740A2
:101C80000300F6F4102FF78EA290F68E0090F68ED9
:101C900002903AE8E866F2F40090F2F5029026F439
:101CA000F40138509D08F3F8A2903D05F3F8A39095
:101CB0003D029A40EE00F3FAA09049A0FD12E00D1B
:101CC000F7FAA1900D0AF09D0892D7404D00F48DCF
:101CD0009236C088DA08C08C08D1C2F5A090405D69
:101CE000EDF2F3F8A29049813D2FE014F6F438901C
:101CF000F6F40A90F2F63890D7404D00F486A43EF0
:101D00002D0FF0465C2420465C3400465C34D740FE
:101D10004D00D444AE3646F462003D02F68E0A9081
:101D2000248F3890F2F4389046F409008DE3F2F4F1
:101D30000A9048413D02E00F0D08E6F41D00B8404E
:101D4000E1E8F7F87D900D01E00FF04F4985EA30AA
:101D5000AE1EE00DE10AD7404D00E4ADA43E808DFB
:101D60008DFAE00DE00EE007F04E5C14E6F5C800D9
:101D70001BD502F40EFED7404D00C474AC3686FE6F
:101D800062008DF2808D8DEEE6F96646E6FA080077
:101D9000D4800400DA087E64F78EA390F78EA590B5
:101DA000F78EA490E00488408840884088408840AE
:101DB000E00CE01BE02AE6F9DF00E0B8DA08FC8B73
:101DC00006F00A00F68E0090F68E02900D023AE8B8
:101DD000E866F2F60090F2F70290F046F05726F42B
:101DE00019003850ED03F3F8A5902DF126F61900EF
:101DF0003870FD0EE118F7F8A390E014D740030007
:101E0000F6F4002FE6F45555D7400300F6F4102FF2
:101E1000F78EA290F68E0090F68E02903AE8E86671
:101E2000F2F40090F2F5029026F4F40138509D0689
:101E3000F3F8A2903D03F3F8A3902DF0F3F8A390EC
:101E400049813D02E00F0D33F3F8A29049813D2E08
:101E5000E014F6F43890F6F40A90F2F63890D74091
:101E60004D00F486A43E2D0FF0465C2420465C34E1
:101E700000465C34D7404D00D444AE3646F44100B1
:101E80003D02F68E0A90248F3890F2F4389046F492
:101E900009008DE3F2F40A9048413D02E06F0D071E
:101EA000E0B4B840E198F7F87D900D01E06FF04F95
:101EB0004986EA303A20E00DE10AD7404D00E4AD12
:101EC000A43E808D8DFAE00DE00EE007F04E5C142C
:101ED000E6F5C8001BD502F40EFED7404D00C474D1
:101EE000AC3686FE62008DF2808D8DEEF78EA0906E
:101EF000E00DE10AD7404D00E4AD9236809D8DFAA9
:101F0000F78EA390F78EA590E00488408840884023
:101F100088408840E00CE01BE02AE6F93300E6F850
:101F20001D00DA08FC8B06F00A00F68E0090F68E93
:101F300002900D023AE8E866F2F60090F2F702909D
:101F4000F046F05726F419003850ED03F3F8A59049
:101F50002DF126F619003870FD0EE118F7F8A39060
:101F6000E014D7400300F6F4002FE6F45555D740AF
:101F70000300F6F4102FF78EA290F68E0090F68EE6
:101F800002903AE8E866F2F40090F2F5029026F446
:101F9000F40138509D08F3F8A2903D05F3F8A390A2
:101FA0003D029A40EE00F3FAA09049A0FD12E00D28
:101FB000F7FAA1900D0AF09D0892D7404D00F48DDC
:101FC0009236C088DA08C08C08D1C2F5A090405D76
:101FD000EDF2F3F8A29049813D2FE014F6F4389029
:101FE000F6F40A90F2F63890D7404D00F486A43EFD
:101FF0002D0FF0465C2420465C3400465C34D7400C
:102000004D00D444AE3646F441003D02F68E0A90AF
:10201000248F3890F2F4389046F409008DE3F2F4FE
:102020000A9048413D02E07F0D08E6F41D00B840EB
:10203000E1B8F7F87D900D01E07FF04F4987EA3075
:102040009A21E00DE10AD7404D00E4ADA43E808D19
:102050008DFAE00DE00EE007F04E5C14E6F5C800E6
:102060001BD502F40EFED7404D00C474AC3686FE7C
:1020700062008DF2808D8DEEE6F96646E6FA080084
:10208000D4800400DA087E64F78EA390F78EA590C2
:10209000F78EA490E0048840884088408840E6F4A9
:1020A00010008840E6FCF800E6FB2200E03AE6F982
:1020B000DF00E0B8DA08FC8B06F00A00F68E00902C
:1020C000F68E02900D023AE8E866F2F60090F2F71A
:1020D0000290F046F05726F419003850ED03F3F85B
:1020E000A5902DF126F619003870FD0EE118F7F8CD
:1020F000A390E014D7400300F6F4002FE6F4555502
:10210000D7400300F6F4102FF78EA290F68E0090C1
:10211000F68E02903AE8E866F2F40090F2F502904A
:1021200026F4F40138509D06F3F8A2903D03F3F82D
:10213000A3902DF0F3F8A29049813D2EE014F6F41F
:102140003890F6F40A90F2F63890D7404D00F486B5
:10215000A43E2D0FF0465C2420465C3400465C34DF
:10216000D7404D00D444AE3646F462003D02F68EB0
:102170000A90248F3890F2F4389046F409008DE3E9
:10218000F2F40A9048413D02E08F0D07E0B4B840F8
:10219000E1D8F7F87D900D01E08FF04F47F8080087
:1021A000EA302A23E00DE10AD7404D00E4ADA43E19
:1021B000808D8DFAE00DE00EE007F04E5C14E6F540
:1021C000C8001BD502F40EFED7404D00C474AC36D7
:1021D00086FE62008DF2808D8DEEF78EA090E00D70
:1021E000E10AD7404D00E4AD9236809D8DFAF78E1E
:1021F000A390F78EA590E0048840884088408840EE
:10220000E6F410008840E6FCF800E6FB2200E03A25
:10221000E6F93300E6F81D00DA08FC8B06F00A0048
:10222000F68E0090F68E02900D023AE8E866F2F61D
:102230000090F2F70290F046F05726F4190038505B
:10224000ED03F3F8A5902DF126F619003870FD0E78
:10225000E118F7F8A390E014D7400300F6F4002F3C
:10226000E6F45555D7400300F6F4102FF78EA290F0
:10227000F68E0090F68E02903AE8E866F2F400904E
:10228000F2F5029026F4F40138509D08F3F8A2907C
:102290003D05F3F8A3903D029A40EE00F3FAA090BA
:1022A00049A0FD12E00DF7FAA1900D0AF09D0892E9
:1022B000D7404D00F48D9236C088DA08C08C08D122
:1022C000C2F5A090405DEDF2F3F8A29049813D2D5A
:1022D000E014F6F43890F6F40A90F2F63890D7400D
:1022E0004D00F486A43E2D0FF0465C2420465C345D
:1022F00000465C34D7404D00D444AE3646F462000C
:102300003D02F68E0A90248F3890F2F4389046F40D
:1023100009008DE3F2F40A9048413D010D06E6F410
:102320001D00B840E1F8F7F87D90A8400806FCFFD2
:10233000FCFEFCFDDB00ECFDECFEECFFF0F9F0E850
:1023400006F066FEE108E4809601E48098015FE80B
:10235000E108E4800400E006F4800400C0855C1518
:10236000E06400400045B864F4800400F1A809A1CD
:10237000E4A0040047FAC8008DEFF78EA690F78E10
:10238000A790E004B840E008E007F0485C14A860BB
:10239000E6F5C8001B6502F40EFED7404D00C4747C
:1023A000AC3686F862008DF1A840F0540851B85060
:1023B00046F509008DE83AE8E866E004B840E10A2D
:1023C000A840D7404D00E4A4A43EA840F0640861B2
:1023D000B86046F609008DF4F2F460904841EA30A6
:1023E000482BD7404E00F3F8850B47F850003D04CA
:1023F000E118E48098010D03E108E4809801F78E6C
:10240000A290F4809801EA204425D7404E00D2F8EB
:102410009E0BDA081676F0D45C4DD7404E00D2F809
:102420009F0BDA081676004D8840D7404E00D2F850
:102430009B0BDA081676F0D45C4DD7404E00D2F8EC
:102440009C0BDA081676004D8840D7404E00D2F833
:10245000980BDA081676F0D45C4DD7404E00D2F8CF
:10246000990BDA081676004D8840D7404E00D2F816
:10247000950BDA081676F0D45C4DD7404E00D2F8B2
:10248000960BDA081676004D8840D7404E00D2F8F9
:10249000920BDA081676F0D45C4DD7404E00D2F895
:1024A000930BDA081676004D8840D7404E00D2F8DC
:1024B0008F0BDA081676F0D45C4DD7404E00D2F878
:1024C000900BDA081676F0C400CDECFCD7404E0035
:1024D000D2F88C0BDA081676F0D45C4DD7404E005B
:1024E000D2F88D0BDA081676F0B400BDECFBD740BD
:1024F0004E00D2F8890BDA081676F0D45C4DD7403E
:102500004E00D2F88A0BDA081676F0A400ADECFA89
:10251000D7404E00D2F8860BDA081676F0D45C4D20
:10252000D7404E00D2F8870BDA081676F094009D5B
:10253000F08EFCFAFCFBFCFCDA08FC8B06F00A00CF
:10254000EA005826D7404E00D2F89B0BDA081676E0
:10255000F0D45C4DD7404E00D2F89C0BDA081676CA
:10256000004D8840D7404E00D2F8980BDA08167616
:10257000F0D45C4DD7404E00D2F8990BDA081676AD
:10258000004D8840D7404E00D2F8950BDA081676F9
:10259000F0D45C4DD7404E00D2F8960BDA08167690
:1025A000004D8840D7404E00D2F8920BDA081676DC
:1025B000F0D45C4DD7404E00D2F8930BDA08167673
:1025C000004D8840D7404E00D2F88F0BDA081676BF
:1025D000F0D45C4DD7404E00D2F8900BDA08167656
:1025E000004D8840D7404E00D2F88C0BDA081676A2
:1025F000F0D45C4DD7404E00D2F88D0BDA08167639
:10260000F0C400CDECFCD7404E00D2F8890BDA08BC
:102610001676F0D45C4DD7404E00D2F88A0BDA081B
:102620001676F0B400BDECFBD7404E00D2F8860B16
:10263000DA081676F0D45C4DD7404E00D2F8870BFE
:10264000DA081676F0A400ADF09FF08EFCFBFCFCDF
:10265000DA08FC8B06F00A00F68E0090F68E0290E7
:102660003AE8E866F48098012D03F3F8A2903D085B
:10267000F2F40090F2F5029026F4370038508DF015
:10268000F68E0090F68E0290F3F8A290EA20C4290C
:102690003AE8E866E004B840A840D7404D00F4842A
:1026A000A43E49823D03E128F7F8A290A8400841E2
:1026B000B840A84046F409008DEFE004B840A840B7
:1026C000D7404D00F484A43E47F878003D0DE12842
:1026D000F7F8A290F68E0090F68E0290E10AA840DC
:1026E000D7404D00E4A4A43EA8400841B840A8400B
:1026F00046F409008DE4E004B840A840D7404D00FE
:10270000F484A43E47F82100EA309A29E128F7F83A
:10271000A290F68E0090F68E0290E10AA840D74073
:102720004D00E4A4A43EE6F86400DA087476F48070
:102730009801EA207028D7404E00D2F89E0BDA08A4
:102740001676F0D45C4DD7404E00D2F89F0BDA08D5
:102750001676004D8840D7404E00D2F89B0BDA0821
:102760001676F0D45C4DD7404E00D2F89C0BDA08B8
:102770001676004D8840D7404E00D2F8980BDA0804
:102780001676F0D45C4DD7404E00D2F8990BDA089B
:102790001676004D8840D7404E00D2F8950BDA08E7
:1027A0001676F0D45C4DD7404E00D2F8960BDA087E
:1027B0001676004D8840D7404E00D2F8920BDA08CA
:1027C0001676F0D45C4DD7404E00D2F8930BDA0861
:1027D0001676004D8840D7404E00D2F88F0BDA08AD
:1027E0001676F0D45C4DD7404E00D2F8900BDA0844
:1027F0001676F0C400CDECFCD7404E00D2F88C0B1E
:10280000DA081676F0D45C4DD7404E00D2F88D0B26
:10281000DA081676F0B400BDECFBD7404E00D2F8D3
:10282000890BDA081676F0D45C4DD7404E00D2F80A
:102830008A0BDA081676F0A400ADECFAD7404E0009
:10284000D2F8860BDA081676F0D45C4DD7404E00ED
:10285000D2F8870BDA081676F094009DF08EFCFA19
:10286000FCFBFCFCDA08FC8B06F00A00EA009A2963
:10287000D7404E00D2F89B0BDA081676F0D45C4DA8
:10288000D7404E00D2F89C0BDA081676004D8840EF
:10289000D7404E00D2F8980BDA081676F0D45C4D8B
:1028A000D7404E00D2F8990BDA081676004D8840D2
:1028B000D7404E00D2F8950BDA081676F0D45C4D6E
:1028C000D7404E00D2F8960BDA081676004D8840B5
:1028D000D7404E00D2F8920BDA081676F0D45C4D51
:1028E000D7404E00D2F8930BDA081676004D884098
:1028F000D7404E00D2F88F0BDA081676F0D45C4D34
:10290000D7404E00D2F8900BDA081676004D88407A
:10291000D7404E00D2F88C0BDA081676F0D45C4D16
:10292000D7404E00D2F88D0BDA081676F0C400CDF1
:10293000ECFCD7404E00D2F8890BDA081676F0D4BA
:102940005C4DD7404E00D2F88A0BDA081676F0B408
:1029500000BDECFBD7404E00D2F8860BDA081676A5
:10296000F0D45C4DD7404E00D2F8870BDA081676CB
:10297000F0A400ADD4500A00F0455C2420455C343E
:1029800000455C34D7404D00D494AC36F08EFCFB4F
:10299000FCFCDA08FC8B06F00A00A840F064086131
:1029A000B86046F60900EA80FA26F2F40090F2F5E3
:1029B000029026F4881338509D05F3F8A2904982BE
:1029C000EA209026F68E6290E014F6F43890E10842
:1029D000E4800200E4800400F3F8A2904981EA3028
:1029E000F02AE108E4809601F2F73890D7404D00D4
:1029F000F487A43E49813D54F48002002D0FE6F691
:102A0000FDFFF4A00400F18A0981E4800400C0A560
:102A10005C15E06400400045B8640D03E118E480F3
:102A20000200F0475C2420475C3400475C34D74008
:102A30004D00D464AC36F4A00400F18A0981E4802E
:102A40000400C0A55C15E06400400045B864E014D3
:102A5000B8403AE8E866A880F0485C14F2F938908B
:102A6000E6F5C8001B9502F40EFED7404D00D46475
:102A7000AC36F4A00400F18A0981E4800400C0A50A
:102A80005C15E06400400045B864F0680861B86017
:102A9000F0495C14D7404D00D454903E40569DD927
:102AA000E10AF2F43890D7404D00E4A4A43E248F0C
:102AB0003890F2F4389046F409008D96E6F6FCFF63
:102AC000F4A00400F1EA09E1E4E00400C0A55C150B
:102AD000E06400400045B864E6FB6800C0EAE068D6
:102AE000008066F8FF3FF2F904FEDA0890740D0DDD
:102AF000F48096010981E4809601E6F82A00DA085C
:102B00009076E6F8FF00DA089679F4809601498518
:102B1000FD05E014F6F40A90F6F46490E014B84071
:102B2000E10AA840D7404E00E4A4820BA840F0641C
:102B30000861B86046F62602FDF4F68E6090E0D893
:102B4000DA089076EA009E2EF2F4249048463D740E
:102B5000F68E2490D7404E00F3F8840B47F83000EF
:102B60003D06E6F81001E6F92000DA08A476D74021
:102B70004E00F3F8840B47F83200EA309E2EF3F84B
:102B80007D9007F8F8FF47F80800EA909E2EC08471
:102B90005C2406F4982B9C04EA00B82BEA00C82BAE
:102BA000EA00D82BEA00E82BEA00F82BEA00082C10
:102BB000EA00182CEA00282CE6F8ED01E6F92000DE
:102BC000DA08A476EA009E2EE6F8D201E6F92000A3
:102BD000DA08A476EA009E2EE6F8B701E6F92000AE
:102BE000DA08A476EA009E2EE6F89C01E6F92000B9
:102BF000DA08A476EA009E2EE6F88101E6F92000C4
:102C0000DA08A476EA009E2EE6F86601E6F92000CE
:102C1000DA08A476EA009E2EE6F84B01E6F92000D9
:102C2000DA08A476EA009E2EE6F83001E6F92000E4
:102C3000DA08A476EA009E2EF68E08903AE8E86656
:102C4000E018DA085E76F2F460903D05E6F41400D0
:102C500042F408909DF3E6F4140042F40890EAE090
:102C60009E2EF78EA290F3FA7D9047FA0C002D0964
:102C700047FA0D002D0647FA0E002D0347FA0F0004
:102C80003D14E0048840884088408840E6F4100005
:102C90008840E6FCF800E6FB2200E03AF09FF08E68
:102CA000DA08FC8B06F00A000D0FE004884088402B
:102CB000884088408840E00CE01BE02AF09FF08EBE
:102CC000DA08FC8B06F00A00F68E0090F68E029071
:102CD0003AE8E866F2F40090F2F5029026F4370044
:102CE00038508DF6F68E0090F68E0290F3F8A29092
:102CF0002D3E3AE8E866E004B840A840D7404D00D1
:102D0000F484A43E49823D03E128F7F8A290A8404C
:102D1000F0640861B86046F609008DEFE004B84041
:102D2000A870D7404D00F487A43E47F878003D0CCA
:102D3000E128F7F8A290F68E0090F68E0290E10A54
:102D4000D7404D00E4A7A43EA840F0840881B88095
:102D500046F809008DE5F2F40090F2F5029026F4B1
:102D6000881338509D04F3F8A29049822DC2F68E44
:102D70006290E014F6F43890E108E4800200E48008
:102D80000400F3F8A29049813D7CE108E4809601BB
:102D9000F2F73890D7404D00F487A43E49813D5466
:102DA000F48002002D0FE6F6FDFFF4A00400F18A86
:102DB0000981E4800400C0A55C15E0640040004582
:102DC000B8640D03E118E4800200F0475C2420475A
:102DD0005C3400475C34D7404D00D464AC36F4A07A
:102DE0000400F18A0981E4800400C0A55C15E06458
:102DF00000400045B864E014B8403AE8E866A880AE
:102E0000F0485C14F2F93890E6F5C8001B9502F41E
:102E10000EFED7404D00D464AC36F4A00400F18A15
:102E20000981E4800400C0A55C15E0640040004511
:102E3000B864F0680861B860F0495C14D7404D0090
:102E4000D454903E40569DD9E10AF2F43890D740D0
:102E50004D00E4A4A43E248F3890F2F4389046F458
:102E600009008D96E6F6FCFFF4A00400F18A0981C2
:102E7000E4800400C0A55C15E06400400045B8642F
:102E80000D05F48096010981E4809601F480960195
:102E90004985FD05E014F6F40A90F6F4649046FEC8
:102EA0001D003D130D0DC2FDA190F09D0892D7406D
:102EB0004D00F48D9236C088DA08C08C258FA19021
:102EC000F3F8A09043F8A190EDEEF2F50A903D04DE
:102ED000F2F46490EA20B62348513D124FE85EE8D0
:102EE000E6F86400DA085E76E6F82A00DA089076FA
:102EF000E6F82100DA089076E0D8DA0890761F40EC
:102F000006F09A01FCFFFCFEFCFDDB00F68E009053
:102F1000F68E0290F68E0A903AE8E866F2F4009097
:102F2000F2F5029026F4370038508DF6F68E0090B8
:102F3000F68E0290F3F8A2902D303AE8E866E007AA
:102F4000D7404D00F487A43E49823D03E128F7F8BD
:102F5000A29080878DF5E007D7404D00F487A43E0E
:102F600047F878003D0CE128F7F8A290F68E009023
:102F7000F68E0290E10AD7404D00E4A7A43E808778
:102F80008DEBF2F40090F2F5029026F4881338509D
:102F90009D04F3F8A29049822DD0F68E6290E01441
:102FA000F6F43890E104E102F3F8A29049813D6122
:102FB000F2F83890D7404D00F488A43E49813D4254
:102FC00049402D0CE6F6E703F1A2F12A0921C0A43D
:102FD0005C14D7404E00C46450000D01E114F04869
:102FE0005C2420485C3400485C34D7404D00D464F5
:102FF000AC36F1A2F12A0921C0A45C14D7404E00DE
:10300000C4645000E0173AE8E866F0475C14F2F94F
:103010003890E6F5C8001B9502F40EFED7404D002F
:10302000D454AC36C0245C14D7404E00C454500075
:1030300008710921F0495C14D7404D00D454903EEA
:1030400040579DE1E10AF2F43890D7404D00E4A4E6
:10305000A43E248F3890F2F4389046F409008DA8ED
:10306000E6F5E603C0245C14D7404E00C45450007B
:10307000DB00D7404E00F68E5000E6F4E603D74062
:103080004E00F6F45200E014F6F40A90DB00ECFD7A
:10309000ECFEECFFF0DCF0EBF0FA88908880280280
:1030A0003AE8E866D4400200F1C8E064D7001400B2
:1030B000B9C4DA08BE57D4400200B840E058DA0874
:1030C0007476D4400400F1C8E064D7001400B9C499
:1030D000DA08BE57D4500400A8400045B840E05874
:1030E000DA087476F06FE064D7001400B9C4DA0827
:1030F000BE57A840004FB840E058DA087476F06E2A
:10310000E064D7001400B9C4DA08BE57A840004EE6
:10311000B840E058DA087476F06DE064D700140027
:10312000B9C4DA08BE57A840004DB840E058DA08E4
:103130007476A85046F5FF00BD0326F50001B8508F
:10314000A840F1C8E064D7001400B9C4DA08BE573B
:10315000F68E2E900806FCFFFCFEFCFDDB00E01462
:10316000F6F4AC90DB00F68EAC90DB00ECFDF68E56
:103170000A90F68E6290F68E6490F68E5890F68ED7
:103180006690F68E6090F68E5690DA08BC423AE869
:10319000E866E0EAE069E018DA082A5FE058DA0851
:1031A0007476E7F8F900F7F89990DA081E44E01809
:1031B000DA087832F0D4DA08BC42F04D49813D5249
:1031C000E6F8DA03E6F92000DA08A476EE905FE884
:1031D000E178F7F87D903AE8E866F2F460904841CB
:1031E0003D05DA08BC42E008DA087832F2F458907B
:1031F00048413D02DA08BC3CF2F4669048413D0289
:10320000DA084641F2F4249048463D1CF68E24909C
:10321000D7404E00F3F8840B47F830003D06E6F83F
:10322000D603E6F92000DA08A476D7404E00F3F87A
:10323000840B47F832003D06E6F8DA03E6F9200091
:10324000DA08A476F2F464903D03F2F40A902DC3F8
:10325000E6F8D303E6F92000DA08A476E0D8DA0825
:1032600090760D03E014F6F40A903FE85EE84EE82D
:10327000DA087264FCFDDB00ECFDECFEECFFF0E82C
:1032800006F0E8FFF78E9D90F78F9E90F78E9F9047
:10329000F78E8B90E108E4800600F04E49813D0BEB
:1032A000F78E8F90E7F8FE00F7F88E90E7F8CA00E7
:1032B000F7F88D900D33D7404E00D2F8860BDA0820
:1032C0001676F0D45C4DD7404E00D2F8870BDA0862
:1032D0001676004DF7F88F90D7404E00D2F8890B44
:1032E000DA081676F0D45C4DD7404E00D2F88A0B3F
:1032F000DA081676004DF7F88E90D7404E00D2F8D7
:103300008C0BDA081676F0D45C4DD7404E00D2F81C
:103310008D0BDA081676004DF7F88D90DA08BA436F
:10332000E108E4800600D7404E00F3FA8E0B47FA1E
:1033300061002D0947FA41002D0647FA70002D0360
:1033400047FA50003D14D7404E00D2F88F0BDA08F0
:103350001676F0D45C4DD7404E00D2F8900BDA08C8
:103360001676004DF7F89E90E118F7F89D90E0046E
:10337000C4400200C4400400C2F48E905C04E00526
:10338000C4400200C4500400F0846880F09566F9DF
:10339000E800C4800200C4900400F0C8F0D9F068CE
:1033A0005C3D5C3C7CD670D6C4C00200C4D0040036
:1033B000F08DE00966F8FF006890F0685C895C8831
:1033C0007C867096F04D7C8466F4FF00685000485F
:1033D000D7400300F6F40C2FF02C66F2FF00F03D0E
:1033E0006830F082F093F0625C895C887C8670962D
:1033F000F04CF05DF06D7C847C855C86704666F4F4
:10340000FF0068500048D7400300F6F40E2FF78EF7
:103410009090E6F4F9FFE6F5EA18C4400A00C450BB
:103420000C00E7F83C00E4800800F3F88D90E4809D
:103430000E00F3F88E90E4800F00F3F88F90E48094
:103440001000E089009066F9FF3FF2FA04FEE018F0
:10345000DA08586AE018DA08406AF68E0090F68EAC
:1034600002903AE8E866F2F40090F2F5029026F451
:10347000C40938509D03F3F890902DF3F68E089010
:10348000F68E0090F68E02900D793AE8E866E00F2D
:103490000D6C3AE8E866F0DF5C3DD7404D00F48DF6
:1034A000C9183D5EF04F5C24D7404D00F48490185D
:1034B000C085F0455C4400455C3420455C24D75011
:1034C0004D00F4A49519F48DC318418AED13E6F864
:1034D000C218E6F94D00008DDA08D445F68E00904A
:1034E000F68E0290058F9490E11AD7404D00E4AD1E
:1034F000C9180D36F04F5C34D7404D00F4C4C818DD
:10350000C0C7D7404D00F427F934F04F5C34D740A2
:103510004D00F484C5184182ED23C02A08A1F04F64
:103520005C34D7404D00F484C418C089F04F5C343B
:10353000D7404D00F484C218C088DA085245F68E90
:103540000090F68E0290F07F5C37D7504D00F4C7A4
:10355000C418F487C518018CD7404D00E487C518FE
:1035600008F146FF0D008D01E00FF04F5C34D740AD
:103570004D00F484C21847F8FF003D8BF3F8949097
:103580004980FD09F2F40090F2F5029026F4581BF0
:103590003850EA808A34F68E0090F68E02900D390B
:1035A0003AE8E866E00F0D2C3AE8E866F06F5C2632
:1035B000D7404D00F48691183D1ED7404D00F4864B
:1035C0009018C085F0455C4400455C3420455C247F
:1035D000D7504D00F4A49519F4868F18418AED0B4D
:1035E000F68E0090F68E0290058F9390E11AD740E8
:1035F0004D00E4A6911808F146FF0D008D01E00F83
:10360000F04F5C24D7404D00F4848E1847F8FF003B
:103610003DCBF3F893904980FD08F2F40090F2F569
:10362000029026F4581B38508DBBF2F4089046F4F3
:1036300064009D04F3F89F90EA208034E00FB8F016
:10364000EA0088383AE8E866F07F5C37D7404D00FA
:10365000F487C9184981EA308638D7404D00F4878D
:10366000C218C085A880F0485C14D7404D00C454EF
:10367000BE10F0480841B840EA0054383AE8E8661D
:10368000D7404D00F427C818C029D7404D00F48911
:103690000635C085F0455C340045E6F51C020B9507
:1036A00002F40EFED7404D00F4848D19C086A84068
:1036B000F0540851B8505C14D7504D00C464BE108B
:1036C000F447C818C04AD7404D00F48A0635C08573
:1036D000F0455C340045E6F51C020BA502F40EFE35
:1036E000D7404D00F4848E19C086A840F05408518C
:1036F000B8505C14D7504D00C464BE10F467C818AD
:10370000C06BD7404D00F48B0635C085F0455C3466
:103710000045E6F51C020BB502F40EFED7404D0045
:10372000F4848F19C086A840F0540851B8505C1436
:10373000D7504D00C464BE10F487C818C08CD74061
:103740004D00F48C0635C085F0455C340045E6F547
:103750001C020BC502F40EFED7404D00F4849019F4
:10376000C086A840F0540851B8505C14D7504D00A2
:10377000C464BE10F487C818C08DD7404D00F48DC6
:103780000635C085F0455C340045E6F51C020BD5D6
:1037900002F40EFED7404D00F4849119C086A84073
:1037A000F0540851B8505C14D7504D00C464BE109A
:1037B000F487C818C084D7404D00F4840635C0850E
:1037C000F0455C340045D7404D00F4A7C818C0A6AA
:1037D000E6F51C020B6502F40EFED7404D00F484A2
:1037E0009219C086A840F0540851B8505C14D750C4
:1037F0004D00C464BE10F487C818C084D7404D0083
:10380000F4840635C085F0455C340045D7404D0052
:10381000F4A7C818C0A6E6F51C020B6502F40EFE5C
:10382000D7404D00F4849319C086A840F054085145
:10383000B8505C14D7504D00C464BE10F487C8184B
:10384000C085D7404D00F48506350981D7404D002D
:10385000E4850635D7404D00F487C818C084D7509A
:103860004D00F4A40635F487C318418AEAE07C369B
:10387000E6F6FFFFA840F0540851B8505C14D7405A
:103880004D00C464BE1008F1F04F5C34D7404D00C9
:10389000F484C21847F8FF002D0446FF0D00EA80AB
:1038A0004436E00FEA00EC3A3AE8E866F07F5C273D
:1038B000D7404D00F48791184981EA30EA3AD74061
:1038C0004D00F4878E18C085A880F0485C14D7405E
:1038D0004D00C454BE10F0480841B840EA00B83A60
:1038E0003AE8E866D7404D00F4279018C029D74041
:1038F0004D00F4890635C085F0455C340045E6F599
:103900001C020B9502F40EFED7404D00F4848D1975
:10391000C086A840F0540851B8505C14D7504D00F0
:10392000C464BE10F4479018C04AD7404D00F48AD2
:103930000635C085F0455C340045E6F51C020BA554
:1039400002F40EFED7404D00F4848E19C086A840C4
:10395000F0540851B8505C14D7504D00C464BE10E8
:10396000F4679018C06BD7404D00F48B0635C085C6
:10397000F0455C340045E6F51C020BB502F40EFE82
:10398000D7404D00F4848F19C086A840F0540851E8
:10399000B8505C14D7504D00C464BE10F487901822
:1039A000C08CD7404D00F48C0635C085F0455C34A2
:1039B0000045E6F51C020BC502F40EFED7404D0093
:1039C000F4849019C086A840F0540851B8505C1493
:1039D000D7504D00C464BE10F4879018C08DD740F6
:1039E0004D00F48D0635C085F0455C340045E6F5A4
:1039F0001C020BD502F40EFED7404D00F484911941
:103A0000C086A840F0540851B8505C14D7504D00FF
:103A1000C464BE10F4879018C084D7404D00F4846D
:103A20000635C085F0455C340045D7404D00F4A70D
:103A30009018C0A6E6F51C020B6502F40EFED740F6
:103A40004D00F4849219C086A840F0540851B85033
:103A50005C14D7504D00C464BE10F4879018C08425
:103A6000D7404D00F4840635C085F0455C340045F0
:103A7000D7404D00F4A79018C0A6E6F51C020B65D0
:103A800002F40EFED7404D00F4849319C086A8407E
:103A9000F0540851B8505C14D7504D00C464BE10A7
:103AA000F4879018C085D7404D00F485063509810C
:103AB000D7404D00E4850635D7404D00F487901877
:103AC000C084D7504D00F4A40635F4878F18418A7E
:103AD000EAE0E038E6F6FFFFA840F0540851B8509D
:103AE0005C14D7404D00C464BE1008F1F04F5C2454
:103AF000D7404D00F4848E1847F8FF002D0446FF90
:103B00000D00EA80A838E00F0D7DF07F5C37007F64
:103B1000D7404D00F4872A19C086A840F084088158
:103B2000B8805C14D7504D00C464BE10F4872B19C4
:103B3000C086F0980891B890F0485C14D7504D00BA
:103B4000C464BE10F4872C19C086F0A908A1B8A0DF
:103B5000F0495C14D7504D00C464BE10F4872D1991
:103B6000C086F0BA08B1B8B0F04A5C14D7504D0026
:103B7000C464BE10F4872E19C086F0CB08C1B8C04B
:103B8000F04B5C14D7504D00C464BE10F4872F195D
:103B9000C086F01C0811B810F04C5C14D7504D00D2
:103BA000C464BE10F4873019C086F0210821B82003
:103BB000F0415C14D7504D00C464BE10F487311935
:103BC000C086F0320831B830F0425C14D7504D0056
:103BD000C464BE10F4873219C086F0D308D1B8D0BF
:103BE000F0435C14D7404D00C464BE10E6F6FFFFFE
:103BF000F05D0851B850F04D5C14D7404D00C464DE
:103C0000BE1008F1C2F59590405FFD0446FF0B0021
:103C1000EA800A3BA8504850FD032851B8500D09CE
:103C2000E118E4800600258F8B90E6F89001DA0811
:103C30007476E6F6FEFFA840F0540851B8505C14C4
:103C4000D7404D00C464BE10F3F8969049813D0200
:103C5000258F8B90F3F8969049813D05F3F88B9072
:103C60004985EA809A32F480060049813D05F3F8DF
:103C70008B904982EA809A32E01FE10AD7404E00D9
:103C8000E4AF820B86FF2502FDF9F04E49803D0C22
:103C9000E6FB6800A8A0E6F8BE10E6F94D00DA08D9
:103CA0009074E0D8DA089076F68E6090F3F89090F1
:103CB00006F01800FCFFFCFEFCFDDB00ECFDECFE5A
:103CC000ECFF06F0EAFFE108B980E6F4FFFFC4402C
:103CD0000200C4400400F78E8C90E00EE10AF06E02
:103CE0005C26D7504D00E4A6AB35E4A6AC3580EE9B
:103CF0008DF5E6F42C52E6F5080088508840E6FB86
:103D0000F9FFE6FCEA18E01AE019E6F8FA00DA082A
:103D1000D8920804E6F400FFE6F5FF00C440020074
:103D2000C4500400E6F400F8E6F5FF07C4400200C2
:103D3000C4500400E6F407FFD7400300F6F4082F50
:103D4000E6F4F800D7400300F6F40A2FE6F4FFFF8C
:103D5000C4400200C4400400E6F4F8FFE6F5FFFFAB
:103D6000C4400200C4500400D7400300F6F50C2FF5
:103D7000E6F4FFF8D7400300F6F40E2FF68E089015
:103D8000E6FF9000EA002E41F04FC08442F4089014
:103D90009D5AF3F88C904980FD56E00E0D4EF04E82
:103DA0005C24D7404D00F484AB353D46D74003003A
:103DB000F2F4002F2EF4D7400300F6F4002FE6F8BB
:103DC0006400DA087476E11AF0DE5C2DD7404D000D
:103DD000E4ADAC35E6FF6400E6F4F9FFE6F5EA1879
:103DE000C4400800C4500A00E7F83C00E480060024
:103DF000D7404D00F48DAA35E4800C00D7404D002B
:103E0000F48DA935E4800D00E108E4800E00E0693E
:103E1000009066F9FF3FF2FA04FEE018DA08586AEB
:103E2000E018DA08406AD7400300F2F4002F784423
:103E3000D7400300F6F4002F08E1C2F58C90405EF5
:103E4000EDAEF68E08903AE8E866F2F458904841F4
:103E5000EA30A03FF68E5890D7404E00D2F8860B3D
:103E6000DA081676F0D45C4DD7404E00D2F8870BB6
:103E7000DA081676004DF7F88F90D7404E00D2F84A
:103E8000890BDA081676F0D45C4DD7404E00D2F894
:103E90008A0BDA081676004DF7F88E90D7404E0060
:103EA000D2F88C0BDA081676F0D45C4DD7404E0071
:103EB000D2F88D0BDA081676004DF148F7F48D90A4
:103EC000F3F28E90C2F38C90F0735C27D7504D00C4
:103ED000E427A935E447AA35E10AD7404D00E4A715
:103EE000AB35E10AD7404D00E4A7AC35E7FAFF0057
:103EF000F0435C34D7604D00E4A4E535E4A4E63536
:103F0000E4A4E735D7604D00E4A4E835E4A4E9353E
:103F1000E4A4EA35D7504D00E4A4EB35E4A4EC3535
:103F2000E004C4400200C4400400C048E009F06856
:103F30005C895C887C867096C024F054E00400485C
:103F40001059C4400200C4500400F3F88C9047F8A4
:103F50000D009D20E004E00588508840D4B00600A4
:103F6000D4C008000832F0A3E019E008DA08D892BB
:103F70000804258F8C90E6F82A00DA089076C2F8BB
:103F80008C902881DA08BC76E0D8DA089076F68E34
:103F900008900D06E6F89303E6F92000DA08A47607
:103FA000F2F466904841EA3008413AE8E866F68E55
:103FB0006690D7404E00F3FA850B47FA45002D7DF9
:103FC00047FA65002D7AE00E0D47F07E5C37D7404A
:103FD0004D00F487E535C086F08E5C38008E5C18A5
:103FE000D7504D00C468BE10F487E635C086D75060
:103FF0004D00C468C010F487E735C086D7504D0027
:10400000C468C210F487E835C086D7504D00C46834
:10401000C410F487E935C086D7504D00C468C61077
:10402000F487EA35C086D7504D00C468C810F487BD
:10403000EB35C086D7504D00C468CA10F487EC3504
:10404000C086D7404D00C468CC10E6F6FFFFD740CD
:104050004D00C468CE1008E1C2F58C90405EEDB50D
:1040600048E0FD17F05E5C3E00E528E1E6F5FEFF66
:10407000F04E5C14D7404D00C454BE1008E1E6FB7E
:104080006800F0AEE6F8BE10E6F94D00DA0890746C
:104090000D10E6F4FEFFD7404D00F6F4BE10E01E12
:1040A000E6FB6800E01AE6F8BE10E6F94D00DA0813
:1040B0009074E0D8DA0890760D27F78E8C90E6FFA2
:1040C0009000F68E0890E00EE10AF06E5C26D75064
:1040D0004D00E4A6AB35E4A6AC3580EE8DF5E00EE0
:1040E000E005F04E5C14D7404D00C454BE1086FE6F
:1040F000E7038DF7D7404E00F78E850BE6F88E0369
:10410000E6F92000DA08A476F2F4609048413D0F09
:10411000F78E8C90E00EE005F04E5C14D7404D0019
:10412000C454BE1086FEE7038DF7E118B980A9805C
:104130003D04F2F46490EA20883D06F01600FCFF8E
:10414000FCFEFCFDDB00ECFDECFEECFFE00EE00F06
:10415000E00DE6F42C52E6F5080088508840E00BAC
:10416000E00CE0FAE019E6F8FA00DA08D892080460
:10417000F06E5C3F5C3E7CD670F6F08FE00966F82E
:10418000FF006890F0685C895C887C867096F04FD0
:104190007C84E00566F4FF0068500048D7400300C7
:1041A000F6F40C2FF08E66F8FF00F09F6890F06830
:1041B0005C895C887C867096F04EF05FF06F7C8442
:1041C0007C855C86704666F4FF0068500048D740E6
:1041D0000300F6F40E2FE00DE10CF04D5C24204DB1
:1041E000D7404D00E4C4133586FD31008DF6E00D57
:1041F000E005F04D5C14D7404D00C454BE1086FD60
:10420000E7038DF7F78E9A90F68E6690F68E0890FB
:104210003AE8E866F2F4089046F4D0078DF9E00D2C
:104220000D1EF05D5C25205DD7404D00F4851535F1
:10423000C086F07D5C27207D5C17D7504D00C46799
:10424000BE10F4851435C086D7404D00C467C01039
:10425000E6F6FFFFD7404D00C467C21008D1F04D0D
:104260005C24204DD7404D00F484133549812DD96D
:1042700048D0FD1028D1E6F6FEFFF04D5C24204D1D
:104280005C14D7404D00C464C21008D1F05D5C2DB1
:1042900020D50D07E6F4FEFFD7404D00F6F4BE1022
:1042A000E01DE6FB6800F0ADE6F8BE10E6F94D0053
:1042B000DA089074FCFFFCFEFCFDDB00DA081A450E
:1042C000F78E8D90F78E8E90F78E8F90F78E909060
:1042D000F78E9690F78E9190F78E9290F78E93903E
:1042E000F78E9490F78E95903AE8E866E008E7FA42
:1042F000FF00D7404D00E4A8853680C88DFAE0085D
:10430000E10AD7404D00E4A8F93480C88DFAE008EE
:10431000E10AD7404D00E4A8063580C88DFAE008D0
:10432000E7FAFF00F0685C26D7404D00E4A68E183F
:10433000E10AD7404D00E4A6911880C88DF1E0084D
:10434000E7FAFF00F0685C36D7404D00E4A6C218DB
:10435000E10AD7404D00E4A6C91880C88DF1E008F5
:10436000E10CF0485C4400485C3420485C24D740B1
:104370004D00E4C49519E009E10EF0495C340049B0
:10438000E6F51C021B8502F40EFED7404D00E4E466
:10439000941986F93B008DF180C88DE23AE8E86611
:1043A000E008E6F5FF00F0485C14D7404D00C45427
:1043B000BE1086F8E7038DF7DB00E6F4DE4AE6F58B
:1043C000080088508840E6FBF9FFE6FCEA18E01A8E
:1043D000E019E6F8FA00DA08D8920804E004E005EB
:1043E00088508840E00BE6FCFF00E0FAE019E008A6
:1043F000DA08D8920804E6F407F8D7500300F6F478
:10440000082FF6F40A2FE6F40740D7400300F6F42D
:104410000C2FE004D7400300F6F40E2FDB00DB0086
:1044200006F0F0FFE10CD7400300F2F5F42F5C55E5
:10443000D7400300F2F4F42F7CB4004566F4FF008B
:10444000F7F89C90F78E9B900D0CC0C4D7404D00A0
:10445000F484853643F89C903D03E118F7F89B906F
:1044600009C1C0C7D7404D00F487853647F8FF0023
:104470002D0647FC0D009D03F3F89B902DE6F3FA03
:104480009D903D06F3F89B903D0347FC0D008D0D7C
:1044900049A13D30F3F89E9043F89C903D2BF3F8F2
:1044A0009B903D2847FC0D009D25F3F89C90D7403C
:1044B0004D00E4878536C086E00776F7EB00E7F825
:1044C0008400B980C4600200C4700400C2F69290F7
:1044D000C2F89190F0580056F075087246F70F0038
:1044E0009D0BF09066F9FF3FF2FA04FEF087DA08C0
:1044F000586A0D02F78F9C90F3F89E9043F89C90B9
:104500003D07F3F89D9049813D03E118F7F89F902E
:10451000F3F89C9006F01000DB00ECFD06F0F0FFD5
:10452000E6F4FFFFC4400200C4400400E02DF09018
:1045300066F9FF3FF2FA04FEF04DC088DA08586AC7
:1045400008D1F04D47F80E00FDF206F01000FCFD1A
:10455000DB0006F0F0FFF048C0845C84F064E00704
:1045600076F7EC1CC2F49990E00570467057F06441
:10457000F075E7F88C00B980C4600200C4500400F4
:10458000E7F81100E4800600F049E4800700F04AF3
:10459000E4800800E7F8FF00E4800900E4800A00F6
:1045A000F3F88D90E4800B00F3F88E90E4800C001B
:1045B000F3F88F90E4800D00F09066F9FF3FF2FA77
:1045C00004FEE018DA08586AE018DA08406A06F0D3
:1045D0001000DB0006F0F0FFDC49A988C0845C8491
:1045E000F064E00776F7EC1CC2F49990E0057046A1
:1045F0007057F064F075E7F88C00B980C460020071
:10460000C4500400E7F81300E4800600DC49F48895
:104610000400E4800700DC49F4880500E480080019
:10462000DC49F4880100E4800900E7F8FF00E48039
:104630000A00F3F88D90E4800B00F3F88E90E4808C
:104640000C00F3F88F90E4800D00F09066F9FF3FC6
:10465000F2FA04FEE018DA08586AE018DA08406A4C
:1046600006F01000DB00F3F8BA9029832D290981A8
:104670003D2EE6F4FDFFD7500300F6F4F02FF2F4E0
:10468000F02F66F4000346F40002EA30DC4AD7401B
:104690000300F2F4F02F66F4000C46F400083D0726
:1046A000E6F4FFF7D7400300F6F4F02F0D02DA0826
:1046B000128AE6F4FFFDD7400300F6F4F02FDB008A
:1046C000E6F4FDFFD7400300F6F4102FDB00E138DD
:1046D00025F8BA90E6F5FDFFC2F1BA90F0915C4979
:1046E000D7500300C459102FD449102F66F400038B
:1046F00046F40002EA30DC4AD7400300D449102FC8
:1047000066F4000C46F400083D33E6F7FF00F0A124
:104710005C1AD7404D00D44A7C3EF0B45C1BF0C11B
:104720005C2C20C15C3C00C15C3CF05B005CD76051
:104730004D00C475AC36C475AE36C475B036D7609E
:104740004D00C475B236C475B436C475B636D7409C
:104750004D00C475B8360847D7404D00C44A7C3E6A
:10476000E6F5FFF7D7400300C459102FEA00CA4A04
:10477000D7400300F489172F67F8F00047F82000AE
:104780003D67D7400300F489182FC087F0C15C1C37
:10479000D7404D00D4AC7C3EF06A5C16F0B15C2B87
:1047A00020B15C3B00B15C3BF086008BD7404D00F4
:1047B000C478AC36D7400300F489192FC087D7409E
:1047C0004D00C478AE36D7400300F4891A2FC08755
:1047D000D7404D00C478B036D7400300F4891B2F72
:1047E000C087D7404D00C478B236D7400300F48963
:1047F0001C2FC087D7404D00C478B436D740030083
:10480000F4891D2FC087D7404D00C478B636D740F5
:104810000300F4891E2FC087D7404D00C478B836F6
:10482000F06A0867D7404D00D44C903E40469D0A40
:10483000E118F7F8A290E11AD7404D00E4A1A43E98
:10484000EA00CA4AD7404D00C46C7C3EEA00CA4A1E
:10485000D7400300F489172F67F8F000EA30964933
:10486000D7400300F489182F47F87F003D12D74046
:104870000300F4891A2F47F878003D0BE7FA780017
:10488000D7404D00E4A1A43EE128F7F8A290EA0049
:10489000CA4AD7400300F489172F67F80F00C08574
:1048A000F0715C17D7404D00C457903EF3F8A090CC
:1048B0004980FD10D7404D00F4819136C086F0410B
:1048C0005C2420415C3400415C34D7404D00C4641A
:1048D000AC360D12D7404D00D4679A3666F6FF000D
:1048E00006F60800F0415C2420415C3400415C3451
:1048F000D7404D00C464AC36D7400300F489182F6C
:10490000C086F0715C2720715C3700715C37D7403E
:104910004D00C467AE36D7400300F489192FC08616
:10492000D7404D00C467B036D7400300F4891A2F32
:10493000C086D7404D00C467B236D7400300F48923
:104940001B2FC086D7404D00C467B436D740030044
:10495000F4891C2FC086D7404D00C467B636D740B7
:104960000300F4891D2FC086D7404D00C467B836B8
:10497000D7400300F4891E2FC086D7404D00C4677E
:10498000BA36E11AD7404D00E4A1A43EE118F7F889
:10499000A290EA00CA4AD7400300F489172F67F8AB
:1049A000F00047F81000EA30CA4AD7400300F48903
:1049B000182FC085F0815C18D7404D00C458903E38
:1049C000F3FEA09049E0FD10D7404D00F4819136F0
:1049D000C086F0415C2420415C3400415C34D74007
:1049E0004D00C464AC360D12D7404D00D4689A36E1
:1049F00066F6FF0006F60800F0415C2420415C34B6
:104A000000415C34D7404D00C464AC36D74003004D
:104A1000F489192FC086F0515C2520515C35005176
:104A20005C35D7404D00C465AE36D7400300F489ED
:104A30001A2FC086D7404D00C465B036D74003005A
:104A4000F4891B2FC086D7404D00C465B236D740CD
:104A50000300F4891C2FC086D7404D00C465B436CE
:104A6000D7400300F4891D2FC086D7404D00C46590
:104A7000B636D7400300F4891E2FC086D7404D00BC
:104A8000C465B836E12AD7404D00E4A1A43EE12830
:104A9000F7F8A290E075D7404D00C4587C3E49E03D
:104AA000FD0AD7404D00F4819136C089E6F81D001B
:104AB000DA08708B0D0AC2F4BA905C14D7404D002E
:104AC000D4949A36E0B8DA08708BE6F5FFFDC2F4AC
:104AD000BA905C44D7400300C454102FDB00F3F8B5
:104AE000BA902981EA202A522982EA206E5009814F
:104AF000EA307C50E6F4FDFFD7400300F6F4F02FD7
:104B00003AE8E866D7400300F2F4F02F66F40003B9
:104B100046F40002EA302A52D7400300F2F4F02FA4
:104B200066F4000C46F400083D0BE118F7F8969087
:104B3000E6F4FFF7D7400300F6F4F02FEA006050E8
:104B4000D7400300F2F5F22F5C55D7400300F2F492
:104B5000F22F7CB4004566F4FF00F7F8BC90C2F673
:104B6000BC90E007F046F057284036F5EE003D08CF
:104B7000E6F4FFFDD7400300F6F4F02FEA006050A2
:104B8000286036F7EA003D08E6F4FFFDD740030051
:104B9000F6F4F02FEA006050F3F28E9043F2BC90EE
:104BA000EA304E4DD7400300F2F5F22F66F50007CC
:104BB0007C35D7400300F2F4F42F7C34004566F4D2
:104BC000FF00F7F8BC90F3F88D9043F8BC902D0BE4
:104BD000F3F8999043F8BC902D06F3F8BC9047F891
:104BE000FF00EA306050E118F7F89090F78EBC9023
:104BF000F78E9B90D7400300F2F5F42F5C55D74019
:104C00000300F2F4F42F7CB4004566F4FF00F7F8DB
:104C10009C900D0EC2F4BC90D7404D00F4848536B4
:104C200043F89C903D03E118F7F89B90258FBC90CA
:104C3000C2F6BC90D7404D00F486853647F8FF0099
:104C40002D08F3F8BC9047F80D009D03F3F89B90F6
:104C50002DE1F3FE9D903D03F3F89B902D0D49E16E
:104C6000EA306050F3F89E9043F89C90EA30605030
:104C7000F3F89B90EA306050F3FA9C90D7404D00D7
:104C8000E4A68536C2F89590F0985C390098D74034
:104C90004D00E4A92A19D7400300F3FCF72FD740B1
:104CA0004D00E4C92B19D7400300F3FCF82FD7407F
:104CB0004D00E4C92C19D7400300F3FCF92FD7406D
:104CC0004D00E4C92D19D7400300F3FCFA2FD7405B
:104CD0004D00E4C92E19D7400300F3FCFB2FD74049
:104CE0004D00E4C92F19D7400300F3FCFC2FD74037
:104CF0004D00E4C93019D7400300F3FCFD2FD74025
:104D00004D00E4C93119D7400300F3FCFE2FD74012
:104D10004D00E4C93219258F9590F3F8959047F826
:104D20000B003D02F78E9590E6F4FFFDD74003009F
:104D3000F6F4F02FF3F89E90418AEA30605049E192
:104D4000EA306050E118F7F89F90EA006050F3F8FD
:104D5000BC9047F8EC00EA306050D7400300F3F80D
:104D6000F72F47F82000EA30824ED7400300F3F8CF
:104D7000FD2F47F8F0009D3ED7400300F3F8FD2FCC
:104D80004182EA306050D7400300F3F8FE2F43F829
:104D90008F90EA306050DA082044C2F891905C2885
:104DA000D7404D00E4888E18D7400300F3FAFA2F5D
:104DB000D7404D00E4A88F18C2F59290C2F49190AC
:104DC0000045F1A8D7504D00E4A89018F4888E183B
:104DD00047F8FF002D07258F9190258F9390E118BC
:104DE000F7F89090E6F4FFFDD7400300F6F4F02FBB
:104DF000EA006050D7400300F3F8FC2F43F88D9091
:104E0000EA306050D7400300F3F8FD2F43F88E904E
:104E1000EA306050D7400300F3F8FE2F43F88F903C
:104E2000EA306050DA082044C2F891905C28D740FC
:104E30004D00E4888E18D7400300F3FAFA2FD740CC
:104E40004D00E4A88F18C2F59290C2F491900045ED
:104E5000F1A8D7504D00E4A89018F4888E1847F8B0
:104E6000FF002D07258F9190258F9390E118F7F87B
:104E70009090E6F4FFFDD7400300F6F4F02FEA002F
:104E80006050D7400300F3F8F72F47F81000EA30DE
:104E90006050D7400300F3F8FD2F47F8F0009D6EF7
:104EA000D7400300F3F8FD2F43F88E90EA306050AE
:104EB000D7400300F3F8FE2F43F88F90EA3060509C
:104EC000DA082044C2F792905C37D7404D00E4875F
:104ED000C218E01AD7400300F3F8FB2FC089D7406F
:104EE0004D00F487C218C088DA085245D740030045
:104EF000F3FAFA2FC2F792905C37D7404D00E4A73F
:104F0000C318D7400300F3FAFB2FD7404D00E4A7A6
:104F1000C418D7400300F3FAFB2FD7404D00E4A795
:104F2000C518C2F59290C2F491900045F1A8D740FF
:104F30004D00E4A7C818D7400300F3FAF82FD74074
:104F40004D00E4A7C618D7400300F3FAF92FD75055
:104F50004D00E4A7C718F487C21847F8FF002D07D3
:104F6000258F9290258F9490E118F7F89090E6F4B1
:104F7000FFFDD7400300F6F4F02F0D72D740030079
:104F8000F3F8FC2F43F88D903D6BD7400300F3F806
:104F9000FD2F43F88E903D64D7400300F3F8FE2FB9
:104FA00043F88F903D5DDA082044C2F792905C3759
:104FB000D7404D00E487C218E01AD7400300F3F849
:104FC000FB2FC089D7404D00F487C218C088DA088B
:104FD0005245D7400300F3FAFA2FC2F792905C379C
:104FE000D7404D00E4A7C318D7400300F3FAFB2FC6
:104FF000D7404D00E4A7C418D7400300F3FAFB2FB5
:10500000D7404D00E4A7C518C2F59290C2F4919024
:105010000045F1A8D7404D00E4A7C818D7400300C9
:10502000F3FAF82FD7404D00E4A7C618D740030085
:10503000F3FAF92FD7504D00E4A7C718F487C21828
:1050400047F8FF002D07258F9290258F9490E11847
:10505000F7F89090E6F4FFFDD7400300F6F4F02F48
:10506000E6F4FFFDD7400300F6F4F02FDB00E6F492
:10507000FDFFD7400300F6F4102FDB00E13825F8E0
:10508000BA90E6F5FDFFC2FCBA905C4CD750030025
:10509000C45C102FD44C102F66F4000346F40002B9
:1050A000EA302A52D7400300D44C102F66F4000C8B
:1050B00046F400083D39E6F5FFF7D7400300C45C2D
:1050C000102FF3F8BA902981F7F8BC90E7FEFF00A3
:1050D000C2F6BC90D7404D00F426F934C029F0A99F
:1050E0005C3A00A9F0B65C4B00B65C3B20B65C2B8A
:1050F000F04A004BD7604D00E4E48D19E4E48E19CA
:10510000E4E48F19D7604D00E4E49019E4E49119C8
:10511000E4E49219D7404D00E4E493190921D74003
:105120004D00E426F9340D7BF3F8BA902981F7F8A5
:10513000BC90D7400300F4AC172F29A1C2FBBC9050
:10514000D7504D00E4ABF934F42BF934C02AF06A9F
:105150005C36006AF09B5C49009B5C39209B5C29B3
:10516000F0860089D7404D00F48894193D50D7400F
:105170000300F4EC182FD7404D00E4E88D19D74018
:105180000300F4EC192FD7404D00E4E88E19C2F467
:10519000BA905C44D7400300F4E41A2FD7404D0086
:1051A000E4E88F19C2F4BA905C44D7400300F4E4F9
:1051B0001B2FD7404D00E4E89019C2F4BA905C442C
:1051C000D7400300F4E41C2FD7404D00E4E89119C8
:1051D000D7400300F4EC1D2FD7404D00E4E89219AE
:1051E000C2F4BA905C44D7400300F4E41E2FD740C9
:1051F0004D00E4E89319E11ED7504D00E4E89419FE
:10520000F48995190981D7404D00E4899519092140
:10521000D7404D00E42BF934E118F7F89090E6F50B
:10522000FFFDD7400300C45C102FDB00E10EF3F854
:10523000BA902981EA2074542981EA306253E6F455
:10524000FDFFD7400300F6F4F02F3AE8E866D740B8
:105250000300F2F4F02F66F4000346F40002EA3093
:105260007454D7400300F2F4F02F66F4000C46F4B7
:1052700000083D07E6F4FFF7D7400300F6F4F02FEF
:105280000D69D7400300F2F5F22F5C55D7400300BB
:10529000F2F4F22F7CB4004566F4FF00F7F8BC90FE
:1052A000F3F2BC9047F2EA002D5547F2EB002D5285
:1052B00047F2EC002D4FC2FC9A90F0AC5C2A20AC77
:1052C000D7404D00E42A1535D7400300F2F5F22F00
:1052D00066F500077C35D7400300F2F4F42F7C34E8
:1052E000004566F4FF00F1C8D7404D00E4CA14350C
:1052F000F78EBC900D18C2F9BC90F0B95C2B20B9A8
:10530000D7504D00F4CB1435F48A1435418C3D0947
:10531000D7504D00F4CB1535F48A1535418C3D013D
:10532000E11E258FBC90F3F89A9043F8BC90FD02E3
:1053300049E02DE149E03D0EE11CD7404D00E4CAB3
:105340001335258F9A90F3F89A9047F83100FD02B3
:10535000F78E9A90E6F4FFFDD7400300F6F4F02FA5
:10536000DB00E13825F8BA90E6F5FDFFC2F8BA9007
:105370005C48D7400300C458102FF3F8BA90298135
:10538000F7F8BC90D7400300D448102F66F4000310
:1053900046F400023D6FD7400300D448102F66F456
:1053A000000C46F400083D0AE6F5FFF7C2F4BC9095
:1053B0005C44D7400300C454102F0D56D74003005F
:1053C000F4A8172FC2FABC90F07A5C37D7404D0092
:1053D000E4A7E535D7400300F4A8182FD7404D00C7
:1053E000E4A7E635D7400300F4A8192FD7404D00B5
:1053F000E4A7E735D7400300F4A81A2FD7404D00A3
:10540000E4A7E835D7400300F4A81B2FD7404D0090
:10541000E4A7E935D7400300F4A81C2FD7404D007E
:10542000E4A7EA35D7400300F4A81D2FD7404D006C
:10543000E4A7EB35D7400300F4A81E2FD7404D005A
:10544000E4A7EC35F06A5C26D7404D00F486AC3515
:105450003D06E11AD7404D00E4A6AB350D05E10A43
:10546000D7404D00E4A6AC35E6F5FFFDD74003007C
:10547000C458102FDB00F3F8BA90298247F80A00CD
:10548000EA901856C0845C2406F48E549C04EA000A
:10549000B654EA00DC54EA00EA54EA001055EA0087
:1054A0003655EA005C55EA008255EA00A855EA0044
:1054B000CE55EA00F455E6F4FDFFD7400300F6F4BC
:1054C000F02FE6F4FFF7D7400300F6F4F02FE6F4F0
:1054D000FFFDD7400300F6F4F02FDB00E6F4FDFFFC
:1054E000D7400300F6F4102FDB00E6F4FDFFD740B1
:1054F0000300F6F4202FE6F4FFF7D7400300F6F49C
:10550000202FE6F4FFFDD7400300F6F4202FDB0048
:10551000E6F4FDFFD7400300F6F4302FE6F4FFF782
:10552000D7400300F6F4302FE6F4FFFDD740030028
:10553000F6F4302FDB00E6F4FDFFD7400300F6F46D
:10554000402FE6F4FFF7D7400300F6F4402FE6F4CF
:10555000FFFDD7400300F6F4402FDB00E6F4FDFF2B
:10556000D7400300F6F4502FE6F4FFF7D7400300CE
:10557000F6F4502FE6F4FFFDD7400300F6F4502F69
:10558000DB00E6F4FDFFD7400300F6F4602FE6F4FD
:10559000FFF7D7400300F6F4602FE6F4FFFDD74095
:1055A0000300F6F4602FDB00E6F4FDFFD7400300B4
:1055B000F6F4702FE6F4FFF7D7400300F6F4702FEF
:1055C000E6F4FFFDD7400300F6F4702FDB00E6F4AD
:1055D000FDFFD7400300F6F4802FE6F4FFF7D74035
:1055E0000300F6F4802FE6F4FFFDD7400300F6F445
:1055F000802FDB00E6F4FDFFD7400300F6F4902F88
:10560000E6F4FFF7D7400300F6F4902FE6F4FFFD31
:10561000D7400300F6F4902FDB00F3F8BA9029820C
:1056200047F80A00EA90BC57C0845C2406F432565E
:105630009C04EA005A56EA008056EA008E56EA00B8
:10564000B456EA00DA56EA000057EA002657EA00A4
:105650004C57EA007257EA009857E6F4FDFFD7402E
:105660000300F6F4F02EE6F4FFF7D7400300F6F45B
:10567000F02EE6F4FFFDD7400300F6F4F02EDB0039
:10568000E6F4FDFFD7400300F6F4102EDB00E6F44D
:10569000FDFFD7400300F6F4202EE6F4FFF7D740D5
:1056A0000300F6F4202EE6F4FFFDD7400300F6F4E5
:1056B000202EDB00E6F4FDFFD7400300F6F4302E89
:1056C000E6F4FFF7D7400300F6F4302EE6F4FFFDD2
:1056D000D7400300F6F4302EDB00E6F4FDFFD740A0
:1056E0000300F6F4402EE6F4FFF7D7400300F6F48B
:1056F000402EE6F4FFFDD7400300F6F4402EDB0019
:10570000E6F4FDFFD7400300F6F4502EE6F4FFF771
:10571000D7400300F6F4502EE6F4FFFDD740030017
:10572000F6F4502EDB00E6F4FDFFD7400300F6F45C
:10573000602EE6F4FFF7D7400300F6F4602EE6F49F
:10574000FFFDD7400300F6F4602EDB00E6F4FDFF1A
:10575000D7400300F6F4702EE6F4FFF7D7400300BD
:10576000F6F4702EE6F4FFFDD7400300F6F4702E39
:10577000DB00E6F4FDFFD7400300F6F4802EE6F4EC
:10578000FFF7D7400300F6F4802EE6F4FFFDD74084
:105790000300F6F4802EDB00E6F4FDFFD7400300A3
:1057A000F6F4902EE6F4FFF7D7400300F6F4902EBF
:1057B000E6F4FFFDD7400300F6F4902EDB00F2F58F
:1057C0000890F68E2E903AE8E866F2F42E90484162
:1057D0009D06F04506F4500042F408909DF4F04513
:1057E00006F4500042F40890ED03E014F6F40A9039
:1057F000DB00ECFDECFEECFFF0E9F0F806F0F8FF62
:10580000E044C4400200E6F42000C4400400E00488
:10581000C44006003AE8E866D4400200D7404E0093
:10582000F484820BD088DA081676F0D45C4DD4402C
:105830000200D7404E00F484830BD088DA08167635
:10584000004DB840F08EDA087476A870F1CEE064AE
:10585000D7001400B9C448F53D07D44006005047AE
:10586000C4400600C440060046FF08002D02DA08C6
:10587000BE57D44006000047C4400600D450020082
:10588000D7404E00F485840BD084C4400400F0451A
:105890000843C4400200D44004003DBCF04F46F42D
:1058A0000900EA90CE595C2406F4AE589C04EA0044
:1058B000E659EA00D258EA00F058EA001C59EA001A
:1058C0005059EA008459EA00A259EA00CE59EA0088
:1058D000E659F08EDA087476D440060066F4FF00CC
:1058E000F1C8E064D7001400B9C4DA08BE570D7BD4
:1058F000D440060066F4FF00C4400600F08EDA08CB
:105900007476D4500600E6F400012045F1C8E06446
:10591000D7001400B9C4DA08BE570D65F08EDA0856
:105920007476D44006007C84F1C8E064D70014008B
:10593000B9C4F08EDA087476D440060066F4FF002D
:10594000F1C8E064D7001400B9C4DA08BE570D4BA3
:10595000F08EDA087476D440060066F4FF00F1C8D1
:10596000E064D7001400B9C4F08EDA087476D4402D
:1059700006007C84F1C8E064D7001400B9C4DA08DA
:10598000BE570D31F08EDA087476D440060066F406
:10599000FF00F1C8E064D7001400B9C4DA08BE57AC
:1059A0000D22D440060066F4FF00C4400600F08ECD
:1059B000DA087476D4500600E6F4FF002045F1C8FA
:1059C000E064D7001400B9C4DA08BE570D0CF08E9D
:1059D000DA087476D4400600F1C8E064D7001400F9
:1059E000B9C4DA08BE5706F00800FCFFFCFEFCFD57
:1059F000DB00ECFDECFEECFFF0D9F0E8E00F3AE85C
:105A0000E866F08EDA087476F04F5C14D7404E00EA
:105A1000D4440000F1C8E064D7001400B9C4F04DCC
:105A200049813D02DA08BE5708F1F04F5C14D740B7
:105A30004E00D444000046F4FFFF2D0346FF28002B
:105A4000CDDEFCFFFCFEFCFDDB007EE06EE0F048FE
:105A5000284146F41300EA907A5B5C2406F4625A0B
:105A60009C04EA00AE5AEA00BA5AEA00C65AEA00B2
:105A70007A5BEA007A5BEA00D25AEA00DE5AEA0070
:105A8000EA5AEA00F65AEA00025BEA000E5BEA0014
:105A90001A5BEA00265BEA00325BEA003E5BEA0042
:105AA0004A5BEA00565BEA00625BEA006E5BE00A72
:105AB000E019E048DA082A5F0D65E00AE029E048CD
:105AC000DA082A5F0D5FE00AE039E048DA082A5F69
:105AD0000D59E00AE069E048DA082A5F0D53E00A50
:105AE000E079E048DA082A5F0D4DE00AE089E048F5
:105AF000DA082A5F0D47E00AE099E048DA082A5FF1
:105B00000D41E00AE0A9E048DA082A5F0D3BE00A0F
:105B1000E0B9E048DA082A5F0D35E00AE0C9E0485C
:105B2000DA082A5F0D2FE00AE0D9E048DA082A5F98
:105B30000D29E00AE0E9E048DA082A5F0D23E00ACF
:105B4000E0F9E048DA082A5F0D1DE0FAE0D9E04804
:105B5000DA082A5F0D17E0FAE0C9E048DA082A5FA0
:105B60000D11E0FAE0B9E048DA082A5F0D0BE0FA1F
:105B7000E079E048DA082A5F0D05E00AE079E048BC
:105B8000DA082A5FE6F86400DA087476DB007EE063
:105B90006EE048903D017FE0F0A9F048D089E048F0
:105BA000DA082A5FE6F86400DA087476DB00ECFDB8
:105BB000ECFEF0C8F0D9F048F059DA08A487F0E418
:105BC000F054BCF5F065DA080088F06CF07DDA0876
:105BD00046883D05F04CF05DDA08A4870D16F04EBE
:105BE000F05EBCF5F065DA080088F064F075F04C02
:105BF000F05DDA082886E006E6F7003FDA08468816
:105C0000CD03F04E08410D01F04EFCFEFCFDDB0023
:105C10003AE8E866E6240000E6F44000F6F4529024
:105C2000D180E6E02A40E6F42A40F6F43C90F68E75
:105C30003A90F68E0090F68E0290E6CB6A003AE833
:105C4000E866F2F43A9048429D0AF2F40090F2F5C8
:105C5000029026F4C40938509D029A40F000E6A450
:105C60001600E6CB0000F2F448FEE005E006DA0894
:105C70000088F064F075F2F40090F2F5029026F4DA
:105C8000C40938508D06E014F6F40A90E004E005EB
:105C9000DB00F046F057DB00ECFDECFEECFFE00D26
:105CA000F68E0A90DA08105CF0E4F0F5E6F462BED5
:105CB000E6F53C3CF06EF07FDA081087F0E4F0F592
:105CC000F084F095DA08AE5BF0D466F400FF7C84D3
:105CD000F6F45A90F04D66F4FF00F6F45C90E0E4C0
:105CE000404DDD09F05D26F50D00F0855C2800854E
:105CF0005C18DA085C8FE00BE08AF2F95C90F2F84D
:105D00005A90DA08C27AF04DFCFFFCFEFCFDDB0085
:105D1000F0A9F048D089E048DA082A5FDB00ECFD02
:105D2000ECFEF0D8E01EE008DA086095E008DA083A
:105D3000BC95E00BE08AE069E008DA08C27A6FE01F
:105D40007EE0E09AE089E048DA082A5FE028DA0895
:105D50007476F68E0090F68E0290F68E2E90E7FC0A
:105D6000FF00E064D7001400B9C43AE8E866F2F432
:105D70002E9048419D07E034E00522F4009032F572
:105D800002909DF3E034E00522F4009032F5029099
:105D9000ED02E00E0D03DA087264E01EF04E498059
:105DA0003D2DE0EAE0D9E048DA082A5FE028DA0889
:105DB0007476F68E0090F68E0290F68E2E90E7FCAA
:105DC000FF00E064D7001400B9C43AE8E866F2F4D2
:105DD0002E9048419D07E034E00522F4009032F512
:105DE00002909DF3E034E00522F4009032F5029039
:105DF000ED02E00E0D03DA087264E02EF04E4980E9
:105E00003D31F05DE138418AED2DE08AE039E0482E
:105E1000DA082A5FE028DA087476F68E0090F68EAB
:105E20000290F68E2E90E7FCFF00E064D70014008D
:105E3000B9C43AE8E866F2F42E9048419D07E03490
:105E4000E00522F4009032F502909DF3E034E00585
:105E500022F4009032F50290ED02E00E0D03DA0814
:105E60007264E03EF04E49803D31F05DE148418A88
:105E7000ED2DE08AE019E048DA082A5FE028DA0828
:105E80007476F68E0090F68E0290F68E2E90E7FCD9
:105E9000FF00E064D7001400B9C43AE8E866F2F401
:105EA0002E9048419D07E034E00522F4009032F541
:105EB00002909DF3E034E00522F4009032F5029068
:105EC000ED02E00E0D03DA087264E04EF04EFCFEC7
:105ED000FCFDDB00ECFEECFFE00EE00FF048C08ABA
:105EE000E009E008DA082A5FE058DA087476E0A8EA
:105EF000DA08DE75F0E4F0F5E006E6F70841DA08C6
:105F00001087DA08A487FCFFFCFEDB003AE8E866AD
:105F1000F04861883A88EA303AE8E8661FEAE6F82D
:105F20003200DA085C8F1EEADB00ECFDECFEECFFD1
:105F3000F0EAF0F9F0D8F04A284146F40F00EA9070
:105F400082615C2406F44A5F9C04EA00865FEA00F2
:105F5000AE5FEA00D65FEA008261EA008261EA0091
:105F6000FE5FEA002660EA004E60EA007660EA0022
:105F70009E60EA00C460EA00EA60EA001061EA009C
:105F80003661EA005C61E008DA080C5FE008DA08D4
:105F90000C5FE008DA080C5FE008DA080C5FE00844
:105FA000DA080C5FE008DA080C5FEA00A661E00896
:105FB000DA080C5FE008DA080C5FE018DA080C5F1A
:105FC000E008DA080C5FE008DA080C5FE008DA089D
:105FD0000C5FEA00A661E008DA080C5FE008DA0866
:105FE0000C5FE008DA080C5FE008DA080C5FE018E4
:105FF000DA080C5FE008DA080C5FEA00A661E00846
:10600000DA080C5FE008DA080C5FE018DA080C5FC9
:10601000E008DA080C5FE018DA080C5FE008DA083C
:106020000C5FEA00A661E008DA080C5FE008DA0815
:106030000C5FE008DA080C5FE008DA080C5FE008A3
:10604000DA080C5FE018DA080C5FEA00A661E008E5
:10605000DA080C5FE018DA080C5FE008DA080C5F79
:10606000E008DA080C5FE008DA080C5FE018DA08EC
:106070000C5FEA00A661E008DA080C5FE008DA08C5
:106080000C5FE008DA080C5FE008DA080C5FE01843
:10609000DA080C5FE018DA080C5FEA00A661E00895
:1060A000DA080C5FE018DA080C5FE008DA080C5F29
:1060B000E008DA080C5FE018DA080C5FE018DA088C
:1060C0000C5F0D71E008DA080C5FE008DA080C5F7D
:1060D000E008DA080C5FE008DA080C5FE008DA088C
:1060E0000C5FE008DA080C5F0D5EE018DA080C5F60
:1060F000E008DA080C5FE008DA080C5FE008DA086C
:106100000C5FE008DA080C5FE008DA080C5F0D4B62
:10611000E008DA080C5FE008DA080C5FE008DA084B
:106120000C5FE018DA080C5FE008DA080C5FE008A2
:10613000DA080C5F0D38E018DA080C5FE008DA08BE
:106140000C5FE008DA080C5FE018DA080C5FE00882
:10615000DA080C5FE008DA080C5F0D25E008DA08C1
:106160000C5FE008DA080C5FE008DA080C5FE00872
:10617000DA080C5FE008DA080C5FE018DA080C5F58
:106180000D12E008DA080C5FE008DA080C5FE0089E
:10619000DA080C5FE008DA080C5FE008DA080C5F48
:1061A000E018DA080C5FF04F284146F40F00EA903F
:1061B000F2635C2406F4BA619C04EA00F661EA002A
:1061C0001E62EA004662EA00F263EA00F263EA0055
:1061D0006E62EA009662EA00BE62EA00E662EA00E7
:1061E0000E63EA003463EA005A63EA008063EA005F
:1061F000A663EA00CC63E008DA080C5FE008DA087E
:106200000C5FE008DA080C5FE008DA080C5FE008D1
:10621000DA080C5FE008DA080C5FEA001664E008B0
:10622000DA080C5FE008DA080C5FE018DA080C5FA7
:10623000E008DA080C5FE008DA080C5FE008DA082A
:106240000C5FEA001664E008DA080C5FE008DA0880
:106250000C5FE008DA080C5FE008DA080C5FE01871
:10626000DA080C5FE008DA080C5FEA001664E00860
:10627000DA080C5FE008DA080C5FE018DA080C5F57
:10628000E008DA080C5FE018DA080C5FE008DA08CA
:106290000C5FEA001664E008DA080C5FE008DA0830
:1062A0000C5FE008DA080C5FE008DA080C5FE00831
:1062B000DA080C5FE018DA080C5FEA001664E00800
:1062C000DA080C5FE018DA080C5FE008DA080C5F07
:1062D000E008DA080C5FE008DA080C5FE018DA087A
:1062E0000C5FEA001664E008DA080C5FE008DA08E0
:1062F0000C5FE008DA080C5FE008DA080C5FE018D1
:10630000DA080C5FE018DA080C5FEA001664E008AF
:10631000DA080C5FE018DA080C5FE008DA080C5FB6
:10632000E008DA080C5FE018DA080C5FE018DA0819
:106330000C5F0D71E008DA080C5FE008DA080C5F0A
:10634000E008DA080C5FE008DA080C5FE008DA0819
:106350000C5FE008DA080C5F0D5EE018DA080C5FED
:10636000E008DA080C5FE008DA080C5FE008DA08F9
:106370000C5FE008DA080C5FE008DA080C5F0D4BF0
:10638000E008DA080C5FE008DA080C5FE008DA08D9
:106390000C5FE018DA080C5FE008DA080C5FE00830
:1063A000DA080C5F0D38E018DA080C5FE008DA084C
:1063B0000C5FE008DA080C5FE018DA080C5FE00810
:1063C000DA080C5FE008DA080C5F0D25E008DA084F
:1063D0000C5FE008DA080C5FE008DA080C5FE00800
:1063E000DA080C5FE008DA080C5FE018DA080C5FE6
:1063F0000D12E008DA080C5FE008DA080C5FE0082C
:10640000DA080C5FE008DA080C5FE008DA080C5FD5
:10641000E008DA080C5F46FE0B00CD04E018DA084D
:106420000C5F0D03E008DA080C5F46FF0B00CD049B
:10643000E018DA080C5F0D03E008DA080C5FE01ED4
:10644000E074204DF0D440DE3D04E018DA080C5F23
:106450000D03E008DA080C5F08E148E6BDF42FEA16
:10646000E018DA0874762EEA3FEAFCFFFCFEFCFD39
:10647000DB00E00AE009E008DA082A5FDB00E6F466
:106480004100D7500300F6F4002FF6F8042FE6F48D
:10649000FFE0D7400300F6F4062FE6F4FFFFD740F5
:1064A0000300F6F4082FE6F4FFF8D7400300F6F4F3
:1064B0000A2FE6F49555D7400300F6F4102FE7F8BD
:1064C0008800D7400300F7F8162FE024D7400300D8
:1064D000F6F4122FE004D7400300F6F4142FE1186D
:1064E000D7400300F7F8172FE138D7400300F7F83B
:1064F000182FE108D7600300F7F8192FF7F81A2FC3
:10650000F7F81B2FD7600300F7F81C2FF7F81D2FA3
:10651000F7F81E2FE6F49955D7400300F6F4202F24
:10652000E108D7400300F7F8262FE6F4FD00D74036
:106530000300F6F4222FE004D7400300F6F4242FE2
:10654000E6F49955D7400300F6F4302FE108D74020
:106550000300F7F8362FE6F4FD20D7400300F6F4E9
:10656000322FE004D7400300F6F4342FE6F49955B7
:10657000D7400300F6F4402FE108D7400300F7F8B6
:10658000462FE6F4FD40D7400300F6F4422FE00426
:10659000D7400300F6F4442FE6F49955D7400300A2
:1065A000F6F4502FE108D7400300F7F8562FE6F431
:1065B000FD60D7400300F6F4522FE004D7400300FB
:1065C000F6F4542FE6F49955D7400300F6F4602F03
:1065D000E108D7400300F7F8662FE6F4FD80D740C6
:1065E0000300F6F4622FE004D7400300F6F4642FB2
:1065F000E6F49955D7400300F6F4702FE108D74030
:106600000300F7F8762FE6F4FDA0D7400300F6F478
:10661000722FE004D7400300F6F4742FE6F4995586
:10662000D7400300F6F4802FE108D7400300F7F8C5
:10663000862FE6F4FDA0D7400300F6F4822FE00495
:10664000D7400300F6F4842FE6F49955D7400300B1
:10665000F6F4902FE108D7400300F7F8962FE6F400
:10666000FDE0D7400300F6F4922FE004D74003008A
:10667000F6F4942FE6F49955D7600300F6F4A02FB2
:10668000F6F4B02FF6F4C02FD7500300F6F4D02F55
:10669000F6F4E02FE108D7400300F7F8E62FE6F420
:1066A000FD00D7400300F6F4E22FE004D7400300DA
:1066B000F6F4E42FE6F49955D7400300F6F4F02FF2
:1066C000E148D7400300F7F8F62FE6F4FFFFD74084
:1066D0000300F6F40C2FE6F4F800D7400300F6F4BC
:1066E0000E2FE6F4C6D7D7400300F6F4F22FE6F4F7
:1066F0008800D7400300F6F4F42F76E54000D74039
:106700000300F2F4022F66F4FFF8D7400300F6F41A
:10671000022FD180E6C36E00F049704A2D04F6F9CD
:10672000B690F6FAB89046F8044E3D07E6F41E001F
:10673000D7400300F6F4002FDB00E0E4D74003006D
:10674000F6F4002FDB00C6030300EC00C687100040
:10675000EC06EC07ECF1ECF2ECF3ECF4ECF5ECF617
:10676000ECF7ECF8ECF9ECFAECFBECFCD7400300AE
:10677000F2F4022F66F4FF00F7F8BA90D740030056
:10678000F2F4002F2EF4D7400300F6F4002F0D4250
:10679000D7400300F2F4002F66F400072D1BD7400A
:1067A0000300F2F4002F66F4000746F400032D0FF7
:1067B000E118F7F8A390E014D7400300F6F4002F97
:1067C000E6F45555D7400300F6F4102F0D03E118F9
:1067D000F7F8A490D7400300F2F4002F9AF409E0F0
:1067E000F3F8A4903D06E6F45555D7400300F6F4BF
:1067F000102FD7400300F2F4022F66F4FF00F7F8E1
:10680000BA90D7400300F2F4002F9AF403B0E118D5
:10681000F7F8A590F3FABA9049A12DBA49A02D0630
:10682000F2F5B890F2F4B690DA080C8AD74003007B
:10683000F2F4002F7844D7400300F6F4002FFCFC5C
:10684000FCFBFCFAFCF9FCF8FCF7FCF6FCF5FCF4AC
:10685000FCF3FCF2FCF1FC07FC06FC87FC00FC03EB
:10686000FB88F048C0845C4426F40A00D74003004B
:10687000F4C4102FDC4AB9C9E002E003F048C08C30
:106880005C4CF04C26F40A00D7400300F484102F2F
:106890009AF43B20F01C26F10C00D7400300D441B1
:1068A000102F66F400F87CB4F064E007E004E00523
:1068B00000261037D7400300D441102F66F4FF00A4
:1068C0005C54E00500241035F048C0845C44F0B40A
:1068D00026FB0E00D7400300D44B102F66F400FFB8
:1068E000E005F0645C555C547CB6705600241035AD
:1068F000D7400300D44B102F66F4FF00E005F0549E
:106900005C55E004002410350D1FF048C0845C4441
:10691000F0B426FB0E00D7400300D44B102F66F4D2
:1069200000E07CD4F064E007E004E005F0270026F6
:10693000F0341037D7400300D44B102F66F4FF001B
:106940005C34E00500241035DC5AC4290200C43947
:106950000400E1020D12F048C0855C45C02BF04BED
:10696000004526F40900D7400300F4E4102FF04955
:10697000004BDC4AE4E406000921F048C0845C4492
:1069800026F40A00D7400300F484102F67F8F000C3
:10699000C085BC45C0244045CDDEF048C0845C4481
:1069A0002841D7400300F4C4102FDC4AE4C90E008C
:1069B000F04847F80F008D0DC0845C4426F41000A9
:1069C000D7400300D444102F66F40C0046F40800AE
:1069D0002D0BE6F5FFFDF048C0845C4426F4100062
:1069E000D7400300C454102FDB00E10CF048C089ED
:1069F0005C49F0A926FA1000D7400300D44A102FB2
:106A000066F4003046F400103D07E6F5FFFBD74082
:106A10000300C45A102FE11CF18CDB00E10AF0489E
:106A2000C0845C4426F41000D7400300D444102FE7
:106A300066F4000346F400023D01E11AF18ADB002E
:106A4000E6F5FFE7F048C0845C4426F41000D74028
:106A50000300C454102FDB00E6F57FFBF048C08B29
:106A60005C4BF04B26F41000D7400300C454102FA9
:106A7000DC4AA9899AF45520DC5AD4490200D45939
:106A8000040066F41F006850F0645CB55CB47C568A
:106A90007056F064F075E004E005F0240026F03450
:106AA0001037DC5AD4490200D459040066F4E01FC0
:106AB0006850F0657C547C555CB6704600241035F7
:106AC000F0CB26FC0C00D7400300C42C102FDC5A5E
:106AD000D4490200D459040066F400E066F51F00B2
:106AE000F0657C547C555CB67046F064F075E0044B
:106AF000E005F0240026F0341037DC5AD4490200B7
:106B0000D4590400684066F5E01FF0457C54E00568
:106B10000024103526FB0E00D7400300C42B102F95
:106B20000D36E005F048C0845C4426F40C00D740E4
:106B30000300C454102FDC5AD4490200D459040075
:106B400068476850F0645CD55CD47C367056F0645D
:106B5000F075E004E005F0240026F0341037DC5A2C
:106B6000D4490200D459040066F4F8076850F0656F
:106B70007C347C355CD6704600241035F048C084E7
:106B80005C4426F40E00D7400300C424102FF048C4
:106B9000C0845C44F0C426FC0A00D7400300F48C97
:106BA000102F9AF43130DC4AA9A977FA0800D740AF
:106BB0000300E4AC102FE10E0D12C0EBF049004BC6
:106BC000DC4AF4C40600F048C0855C45F04B004543
:106BD00026F40900D7400300E4C4102F09E1DC4A81
:106BE000A98967F8F000C085BC45C0E44045CDE503
:106BF000E6F5BFF6F048C0845C4426F41000D740A8
:106C00000300C454102F0D13DC4AA9A967FAF7003A
:106C1000D7400300E4AC102FE6F5BFF7F048C0847E
:106C20005C4426F41000D7400300C454102FDC4A03
:106C3000F4A90E00F048C0845C442841D74003000A
:106C4000E4A4102FDB00E6F5FFFAF048C0845C44B2
:106C500026F41000D7400300C454102FE1020D0E9B
:106C6000DC4A99C9F048C0855C45C024004526F43B
:106C70000900D7400300E4C4102F0921F048C08464
:106C80005C4426F40A00D7400300F484102F67F810
:106C9000F000C085BC45C0244045CDE2E6F5FFF7D5
:106CA000F048C0845C4426F41000D7400300C4546C
:106CB000102FDB00ECFF0EFFF048C0875C47F09719
:106CC00026F91000D7400300D449102F66F4000CB9
:106CD00046F400083D07E6F5FFF7D7400300C45926
:106CE000102F0FFF4AFFF4006981FCFFDB00ECFF6F
:106CF0000EFFF048C0875C47F09726F91000D74098
:106D00000300D449102F66F400A23D07E6F57FFF8B
:106D1000D7400300C459102F0FFF4AFFF4006981C8
:106D2000FCFFDB00E6F5FFFDF048C0845C4426F480
:106D30001000D7400300C454102FDB006EE6E018AB
:106D4000DA0874766FE6E018DA087476F68E7490D6
:106D50001EE2D180E65818023AE8E866F2F4749030
:106D60002DFB1FE2F2F4B2F0DB0006F0D8FFE006E4
:106D7000E005F0465C14D7404E00C45450008096A5
:106D8000CDF8F68E7290F68E0A90F68E74901EE212
:106D9000F0495C8406F41700F6F4B0F03AE8E866CF
:106DA000F2F474902DFB1FE2F2F4B2F0C440020042
:106DB000F68E74901EE2F04A5C840844F6F4B0F05B
:106DC0003AE8E866F2F474902DFB1FE2F2F4B2F0B8
:106DD000C4400400F68E74901EE2F04B5C840844BC
:106DE000F6F4B0F03AE8E866F2F474902DFB1FE296
:106DF000F2F4B2F0C4400600F68E74901EE24884AD
:106E00003D07F04C5C8406F40C00F6F4B0F00D0580
:106E1000F04C5C840844F6F4B0F03AE8E866F2F42A
:106E200074902DFB1FE2F2F4B2F0C44008004884D5
:106E3000EAB0F66FF68E74901EE248853D08D440A5
:106E400028005C8406F40C00F6F4B0F00D06D44083
:106E500028005C840844F6F4B0F03AE8E866F2F4FE
:106E600074902DFB1FE2F2F4B2F0C4400A00488592
:106E7000EAB0F66FF68E74901EE248863D08D44064
:106E80002A005C8406F40C00F6F4B0F00D06D44041
:106E90002A005C840844F6F4B0F03AE8E866F2F4BC
:106EA00074902DFB1FE2F2F4B2F0C4400C0048864F
:106EB000EAB0F66FF68E74901EE248873D08D44023
:106EC0002C005C8406F40C00F6F4B0F00D06D440FF
:106ED0002C005C840844F6F4B0F03AE8E866F2F47A
:106EE00074902DFB1FE2F2F4B2F0C4400E0048870C
:106EF000EAB0F66FF68E74901EE246F808003D0880
:106F0000D4402E005C8406F40C00F6F4B0F00D06BC
:106F1000D4402E005C840844F6F4B0F03AE8E86609
:106F2000F2F474902DFB1FE2F2F4B2F0C4401000B2
:106F300046F80800BD60F68E74901EE246F809001F
:106F40003D08D44030005C8406F40C00F6F4B0F048
:106F50000D06D44030005C840844F6F4B0F03AE802
:106F6000E866F2F474902DFB1FE2F2F4B2F0C44034
:106F7000120046F80900BD3FF68E74901EE246F8F6
:106F80000A003D08D44032005C8406F40C00F6F49C
:106F9000B0F00D06D44032005C840844F6F4B0F042
:106FA0003AE8E866F2F474902DFB1FE2F2F4B2F0D6
:106FB000C440140046F80A00BD1EF68E74901EE20E
:106FC00046F80B003D08D44034005C8406F40C0005
:106FD000F6F4B0F00D06D44034005C840844F6F4B6
:106FE000B0F03AE8E866F2F474902DFB1FE2F2F498
:106FF000B2F0C4401600F68E08903AE8E866E6F46F
:10700000640042F408908D03F2F472902DF6F68E2F
:1070100074901EE2D180E65802003AE8E866F2F485
:1070200074902DFB1FE2F2F4B2F0C4401800D4407B
:10703000180006F02800DB00E017F68E7290F68E3E
:107040000A90F68E74901EE2D180E65802003AE86B
:10705000E866F2F474902DFB1FE2F2F5B2F048718D
:107060003D09F04566F4FF0046F448002D03E014A6
:10707000F6F40A9048723D09F04566F4FF0046F4C4
:107080006B002D03E014F6F40A90F06566F6FF003D
:10709000D7404E00F2F4500000475C14D7404E0039
:1070A000C4645000087146F70E00DD06F04566F432
:1070B00000E046F400402DC5F2F40A903D13E6F6D8
:1070C000E703D7404E00F2F4500000475C14D7505D
:1070D0004E00C4645000F2F450000047D7404E0008
:1070E000F6F45000DB00ECFDECFEECFF2804E04E73
:1070F000E6F42000B840E108E48002001FE2D180FD
:10710000E6E0AA0AE014F6F45690F68E6490F68E45
:107110006290F68E0A90F68E7290DA087097E00A06
:10712000E029E038DA082A5FDA083C6DE00488409C
:10713000884088408840884088408840E01CE6FBC2
:10714000F100E6FA6A00E6F96800E058DA086A6DCC
:1071500006F00E0066F4300046F430002D03E01413
:10716000F6F40A90F68E7290F68E0A90F68E0090E3
:10717000F68E02903AE8E866F2F4729048413D0BD0
:10718000DA083870F2F40A903D04F68E0090F68E1C
:107190000290F68E0A90F2F40090F2F5029026F436
:1071A000C80038508DE7D7404E00F2F4580066F41E
:1071B000FF0046F441002D03E014F6F40A90F2F4C7
:1071C0000A90EA308674E6F83000E6F92000DA0822
:1071D000A476EE905FE8E168F7F87D903AE8E8661B
:1071E000E014F6F45690F2F460904841EA30FE73F1
:1071F000F2F40A90EA30FE73F68E6090E04EE6F408
:107200002000B840E00F3AE8E866D7404E00F48E20
:10721000820BD088DA081676F0D45C4DD7404E0049
:10722000F48E830BD088DA081676004DF1A8D7408B
:107230004E00E4AFB80AD7404E00F48E840BD084E1
:10724000B84008F108E3A8403DDEF68E7290DA08F7
:107250003C6DF68E0090F68E0290D7404E00F68E72
:1072600050003AE8E866F2F4569048413D45D74070
:107270004E00C2F4C20A8840D7404E00C2F4C10A90
:107280008840D7404E00C2F4C00A8840D7404E0024
:10729000C2F4BF0A8840D7404E00C2F4BE0A8840FC
:1072A000D7404E00C2F4BD0A8840D7404E00C2F419
:1072B000BC0A8840D7704E00C2FCBB0AC2FBBA0AA7
:1072C000C2FAB90AC2F9B80AF08FDA086A6D06F094
:1072D0000E0066F4300046F430002D03E014F6F49E
:1072E0000A90F2F40A903D02F68E5690F68E729055
:1072F000F68E0090F68E0290F2F4729048413D0BAB
:10730000DA083870F2F40A903D04F68E0090F68E9A
:107310000290F68E0A90F2F40090F2F5029026F4B4
:10732000960038508D9ED7404E00F2F450002D3616
:10733000E108E4800200E01EE6F82A00DA08907610
:107340003AE8E866F0DE5C1DD7404E00D44D5000B0
:1073500046F4E7033D05E6F82600DA0890760D0AC4
:10736000D7404E00D48D5000DA089679E6F8200018
:10737000DA089076E005F04E5C14D7404E00C45415
:10738000500008E1D7404E00F2F550002851405E11
:107390009DD7D7404E00F68E50000D19F4800200A4
:1073A0000981E4800200E6F82A00DA089076E6F81F
:1073B000FF00DA089679F48002004985FD06E014A2
:1073C000F6F40A90F6F462900D02F68E0A90E01E32
:1073D000E10AD7404E00E4AE820B86FE2502FDF99D
:1073E000E01EE005F04E5C14D7404E00C45450003F
:1073F00086FE2502FDF7E0D8DA0890760D2AF2F431
:10740000249048463D1DF68E2490D7404E00F3F858
:10741000840B47F830003D06E6F82C00E6F9200022
:10742000DA08A476D7404E00F3F8840B47F8320010
:107430003D10E6F83000E6F92000DA08A4760D09E0
:10744000F2F4649048413D05E014F6F46290F68E43
:107450006490F2F46290EA20DC71F2F40A90484100
:107460003D124FE85EE8E6F86400DA085E76E6F87A
:107470002A00DA089076E6F82100DA089076E0D85B
:10748000DA0890761F400804FCFFFCFEFCFDDB00E0
:10749000ECFDECFEECFFF0DB88A0F0E8F0F9280250
:1074A000E6F82A00DA089076E004B840EA00C875E9
:1074B000F04D47F848002D0347F868003D38A860B4
:1074C0005C16F04E0046DC4FA84446F4FFFF2D0941
:1074D000A8605C16F04E0046DC4FA84446F4FDFF61
:1074E0003D05E6F82600DA0890760D58A8605C168F
:1074F000F04E0046DC4FA84446F4FEFF3D05E6F89A
:107500002300DA0890760D4AA8605C16F04E00461B
:10751000DC4FA84446F4FCFF2D41A8605C16F04EF9
:107520000046DC4FA844C088DA0896790D37A86079
:107530005C16F04E0046DC4FA84446F4FFFF2D09D0
:10754000A8605C16F04E0046DC4FA84446F4FDFFF0
:107550003D05E6F82600DA0890760D20A8605C1656
:10756000F04E0046DC4FA84446F4FEFF3D05E6F829
:107570002300DA0890760D12A8605C16F04E0046E3
:10758000DC4FA84446F4FCFF2D09A8605C16F04EC1
:107590000046DC4FA844C088DA08BC76D45002000C
:1075A0002852A8404054FD0DA8605C16F04E0046DD
:1075B000DC4FA84446F4FDFF2D04E6F82000DA086D
:1075C0009076A8400841B840D4500200A8404045F9
:1075D000EA80B0740804FCFFFCFEFCFDDB007ECCFE
:1075E000F68E1490F04806F48000F6F4A0FF3AE816
:1075F000E866F2F414902DFBF2F4A0FE66F4FF03AB
:10760000E005E006DA080088E6F68941E6F79C40E6
:10761000DA081087DB00F04847F83000CD0747F85C
:107620003900AD04D08426F43000DB00F04847F880
:107630006100CD0747F86600AD04D08406F4A9FFC9
:10764000DB00F04847F84100CD0747F84600AD049D
:10765000D08406F4C9FFDB00E6F43000DB00F2F66C
:107660000890F0480046F0543AE8E86642F5089081
:107670009DFBDB00F68E0090F68E02903AE8E866FD
:10768000F048E00522F4009032F502909DF7DB000F
:10769000D1807ECEF048D084F6F4B0FED1809ACE70
:1076A000FD70DB00F0A8F0B90D05DC4B998AD0889D
:1076B000DA089076DC4BA98A3DF8DB0006F0F4FF8F
:1076C000E6F41027F6F80EFE5B44F2F60EFEC460F8
:1076D00002001B64F2F50EFEF0682065E6F4E80394
:1076E000F6F60EFE5B44F2F70EFEC4700400F0578F
:1076F000F0755C5520575C2500575C352065E6F435
:107700006400F6F60EFE5B44F2F70EFEC47006004F
:10771000F057F0755C2520575C3500575C252065D7
:10772000E0A4F6F60EFE5B44F2F70EFEC47008000D
:10773000F057F0755C2500575C15F0462045C440B5
:107740000A00E006E015F0855C18F010F091009852
:10775000A8A948A0ED05D4400A003D0348553D01C5
:10776000E01648613D0CF04A06F43000F1E8D180A3
:107770007ECED0E4F6F4B0FED1809ACEFD70805576
:10778000CDE206F00C00DB00F0A8F0B906F0D4FF63
:10779000E6F600CAE6F79A3BF048F059DA08448961
:1077A000F084F095C4400400C4500600E6F600CA18
:1077B000E6F79A3BDA082C89F084F09520A430B5DE
:1077C000E6F600E1E6F7F505F04AF05BDA084489F1
:1077D000F084F095C4400800C4500A00E6F600E1C9
:1077E000E6F7F505DA082C89F084F09520A430B589
:1077F000E6F68096E6F79800F04AF05BDA084489EE
:10780000F084F095C4400C00C4500E00E6F680965B
:10781000E6F79800DA082C89F084F09520A430B5BA
:10782000E6F64042E0F7F04AF05BDA084489F0847B
:10783000F095C4401000C4501200E6F64042E0F754
:10784000DA082C89F084F09520A430B5E6F6A086FD
:10785000E017F04AF05BDA084489F084F095C44000
:107860001400C4501600E6F6A086E017DA082C894A
:10787000F084F09520A430B5E6F61027E007F04A32
:10788000F05BDA084489F084F095C4401800C450D5
:107890001A00E6F61027E007DA082C89F084F09544
:1078A00020A430B5E6F6E803E007F04AF05BDA081A
:1078B0004489F084F095C4401C00C4501E00E6F6D4
:1078C000E803E007DA082C89F084F09520A430B5AD
:1078D000E6F66400E007F04AF05BDA084489F084D9
:1078E000F095C4402000C4502200E6F66400E00792
:1078F000DA082C89F084F09520A430B5E0A6E007E2
:10790000F04AF05BDA084489F084F095C440240022
:10791000C4502600E0A6E007DA082C89F084F09530
:10792000F04A2048F05B3059C4402800C4502A0077
:10793000E008E009E016F0A65C2AF010F0B100BA09
:10794000A82BD43B0200F042F05328403850ED09F8
:10795000D4402800D4502A0070453D0546F60A0060
:107960003D02E018E009F048F059284138503D0E3A
:10797000F04206F43000F0531850F1E8D1807ECE8A
:10798000D0E4F6F4B0FED1809ACEFD7080A6CDD3BF
:1079900006F02C00DB00F068F048BC347CC4F058E2
:1079A0000054BC4546F50900ED0306F530000D0214
:1079B00006F53700F085DA089076E6F41000F6F662
:1079C0000EFE4B44F2F50CFEF2F70EFE46F50900F2
:1079D000ED0306F530000D0206F53700F085DA08F4
:1079E0009076DB00ECFDECFEF0D9F0E8DA082890A8
:1079F000F04EC088DA0842908A40FE409A40045017
:107A0000DA08968FE1180D0FF04DC088DA08429021
:107A10008A40FE409A400450DA08968FE1180D0320
:107A2000DA08968FE108FCFEFCFDDB00ECFDF0D8E7
:107A30003AE8E866DA082890F04DC0880881DA084C
:107A400042908A40FE409A400450DA08968FE1182E
:107A50000D0EE028DA085C8FE018DA0880908A4082
:107A6000FE40F3F800F8F0D4DA08968FF04DFCFDF4
:107A7000DB00ECFDECFEF0E9F0D8F048C088DA0855
:107A80002C7A704ED089F04DC088DA08E479FCFE7B
:107A9000FCFDDB00ECFDECFEF0D9F0E8F048C0881E
:107AA000DA082C7AF1A8E7F8FF00204DF0D4F18A2B
:107AB000604DD089F04EC088DA08E479FCFEFCFD08
:107AC000DB007EE6E7FC1500E044D7001400B9C4F3
:107AD00046FA08003D2848B03D06E7FC9300E00464
:107AE000D7001400B9C448B13D06E7FC8700E004A4
:107AF000D7001400B9C448B23D06E7FC8300E00497
:107B0000D7001400B9C448B33D06E7FC8B00E0047D
:107B1000D7001400B9C448B43D06E7FC8F00E00468
:107B2000D7001400B9C448A73D2848B03D06E7FC7B
:107B30009200E004D7001400B9C448B13D06E7FC48
:107B40008600E004D7001400B9C448B23D06E7FC43
:107B50008200E004D7001400B9C448B33D06E7FC36
:107B60008B00E004D7001400B9C448B43D06E7FC1C
:107B70008F00E004D7001400B9C4E15CE044D700F2
:107B80001400B9C4E7FCDD00E024D7001400B9C438
:107B9000E7FC6F00E084D7001400B9C4E14CE0A416
:107BA000D7001400B9C4F068E0C4D7001400B9C409
:107BB000F069E0E4D7001400B9C4E7FC8500E044B4
:107BC000D7001400B9C4DB00C6030300EC00C6876D
:107BD0001000EC06EC07ECF1ECF2ECF3ECF4ECF555
:107BE000ECF6ECF7ECF8ECF9ECFAECFBECFCECFD69
:107BF0007EB7F2F4B2FEF0D4F04D47F82A003D040F
:107C0000F68E2290EA00E481F04D47F80D00EA304C
:107C1000D281E10AF2F72290D7404E00E4A7820B0E
:107C2000E10AD7404E00E4A7830BE10AD7504E008B
:107C3000E4A7840BF3F8820B07F8CA00EA20AE7EB3
:107C40002983EA204C810987EA30E481D7404E003D
:107C5000F3F8830B07F8D0FF47F80A00EA90E481B5
:107C6000C0845C2406F46A7C9C04EA00927CEA00EE
:107C7000507EEA00647EEA00787EEA00787EEA00C0
:107C8000787EEA00787EEA00787EEA00787EEA0074
:107C9000827ED7504E00F78E820BF3F8840B07F8E4
:107CA000CF002D2C29822D3729812D4229832D4F5C
:107CB00029828D562D5E07F8F8002D602981EA2073
:107CC000D67D2984EA20FA7D07F8E5002D57298121
:107CD000EA20D67D2984EA20FA7D07F83600EA30CA
:107CE000E481E6F82A00DA089076F2F80490DA08DF
:107CF000BC76E0D8DA089076EA00E481E6F82A005B
:107D0000DA089076F2F80690DA08BC76E0D8DA085D
:107D10009076EA00E481E6F82A00DA089076F2F834
:107D20000C90DA08BC76E0D8DA089076EA00E481B4
:107D30003AE8E866E6F82A00DA089076F2F8169053
:107D4000DA08BC76E0D8DA089076EA00E481E6F852
:107D50002A00DA089076E0D8DA089076EA00E48122
:107D6000E6F82A00DA089076E0D8DA089076EA0099
:107D7000E481E094F6F42A90EA00E481F3F88A9032
:107D800067F80F00D08428422D0E28428D142D1B39
:107D90000843EA30E481E6F88503E6F92000DA08D2
:107DA000A476EA00E481E6F87F03E6F92000DA0829
:107DB000A476EA00E481E6F87603E6F92000DA0822
:107DC000A476EA00E481E6F87003E6F92000DA0818
:107DD000A476EA00E4819AE008E0E6F86A03E6F9AE
:107DE0002000DA08A476EA00E481E6F85E03E6F90A
:107DF0002000DA08A476EA00E481E6F82A00DA082E
:107E00009076E00DF04DD084D7402000F4845203EA
:107E1000D088DA08907608D1F04D47F80B00BDF213
:107E2000E6F82000DA089076E00DF04DD084D740D7
:107E30002000F4844903D088DA08907608D1F04D08
:107E400047F80800BDF2E0D8DA089076EA00E4814D
:107E5000D7404E00F3F8840B0D00E024F6F4249094
:107E6000EA00E481D7404E00F3F8840B0D00E024D3
:107E7000F6F42490EA00E481E024F6F42490EA0089
:107E8000E481D7404E00F3F8840B07F8C7FF3D0AA2
:107E9000E6F82A00DA089076E024F6F42C90E0D890
:107EA000DA089076E024F6F42490EA00E481D740E2
:107EB0004E00F3F8830B07F8D0FF47F80A00EA906A
:107EC000E481C0845C2406F4CC7E9C04EA00F47E49
:107ED000EA001A81EA001A81EA001A81EA001A818E
:107EE000EA001A81EA001A81EA001A81EA001A817E
:107EF000EA002281D7504E00F78E820BF3F8840BF4
:107F000007F8CF002D2E29822D3929822D44298270
:107F10008D472D4B29828D4F2D5307F8F8002D5595
:107F200029828D64EA2030802983EA204C8007F87A
:107F3000E5002D4B29828D5A2D7B2983EA204C8028
:107F400007F83600EA30E481E6F82A00DA0890768D
:107F5000F2F80490DA08BC76E0D8DA089076EA0005
:107F6000E481E6F82A00DA089076F2F80690DA085A
:107F7000BC76E0D8DA089076EA00E481E6F82A00D8
:107F8000DA089076F2F80C90DA08BC76E0D8DA08D5
:107F90009076EA00E481E014F6F46690EA00E48169
:107FA000E014F6F45690EA00E481E014F6F46490EC
:107FB0000F40EA00E481E014F6F46090EA00E48106
:107FC000E014F6F45890EA00E481DA089E92E6F8AC
:107FD0002A00DA089076F2F8AE90F2F9B090DA085A
:107FE0008877E0D8DA089076EA00E481E6F82A009B
:107FF000DA089076D7404E00F3FA850B47FA430033
:108000002D0347FA63003D08E024D7000F00A84481
:10801000F084DA08BC760D07E004D7000F00A8440E
:10802000F084DA08BC76E0D8DA089076EA00E481D9
:10803000DA085E31E6F82A00DA089076E018DA0805
:10804000BC76E0D8DA089076EA00E481F3FA7D9015
:108050002D5829A22D1829A22D1E29A22D2429A28E
:108060008D492D2929A28D2F2D3629A12D3C07FAC6
:108070000A00EA30E481E6F83503E6F92000DA0880
:10808000A476EA00E481E6F81E03E6F92000DA08A7
:10809000A476EA00E481E6F80203E6F92000DA08B3
:1080A000A476EA00E481E6F8E602E6F92000DA08C0
:1080B000A476EA00E481E6F8CB02E6F92000DA08CB
:1080C000A476EA00E481E6F8B002E6F92000DA08D6
:1080D000A476EA00E481E6F89502E6F92000DA08E1
:1080E000A476EA00E481E6F87A02E6F92000DA08EC
:1080F000A4760D78E6F86B02E6F92000DA08A4769B
:108100000D71E6F82A00DA089076C2F87C90DA0859
:10811000BC76E0D8DA0890760D65E064F6F4249039
:108120000D61D7404E00F3F8840B07F8C7FF3D0AF6
:10813000E6F82A00DA089076E024F6F42C90E0D8ED
:10814000DA089076E064F6F424900D4CD7404E00A7
:10815000F3F8830B07F8D0FF47F80A009D43C0846B
:108160005C2406F468819C04EA009081EA009E8108
:10817000EA009E81EA009E81EA009E81EA009E81DB
:10818000EA009E81EA009E81EA009E81EA00A681C3
:10819000D7504E00F78E820BF3F8840B0D23E0943A
:1081A000F6F424900D1FD7404E00F3F8840B07F827
:1081B000C7FF3D0BE6F8A4FFDA089076E0D8DA08AE
:1081C0009076E6E30000FA000000E094F6F42490D4
:1081D0000D09F06DF2F52290248F2290D7404E00C9
:1081E000E4C5820BFCFDFCFCFCFBFCFAFCF9FCF892
:1081F000FCF7FCF6FCF5FCF4FCF3FCF2FCF1FC07EC
:10820000FC06FC87FC00FC03FB88F68E0A90D180FC
:10821000E6E0AA0AE0AAE029E028DA082A5F6EE68A
:10822000E018DA0874766FE6F68E7690E10CE6F4E4
:108230002A00D7001500B9C4E6F42200D7001500C3
:10824000B9C4E6F42300D7001500B9C4E6F424004D
:10825000D7001500B9C4E7FCFF00E6F42500D700FD
:108260001500B9C4E6F42600D7001500B9C4E6F439
:108270002700D7001500B9C43AE8E866E10CE6F437
:108280002100D7001500B9C43AE8E866E7FCF10020
:10829000E6F42B00D7001500B9C4E7FC6B00E6F448
:1082A0002D00D7001500B9C43AE8E866E7FC610084
:1082B000E004D7001500B9C4E7FC6A00E014D70059
:1082C0001500B9C4E11CE034D7001500B9C4E10CB5
:1082D000E044D7001500B9C43AE8E866E7FC6A0054
:1082E000E6F42C00D7001500B9C4E15CE6F41300F5
:1082F000D7001500B9C4E10CE6F42100D700150041
:10830000B9C4F68E0090F68E02903AE8E866F2F470
:1083100076903D08E6F43200E00522F4009032F554
:1083200002909DF3E6F43200E00522F4009032F56D
:108330000290ED06E014F6F40A903AE8E866DB00F5
:10834000E6F42300D7001500A9C4F68E7690E10C60
:10835000D7001500B9C4E6F42200D7001500B9C44F
:10836000E6F42400D7001500B9C4E6F42100D700D4
:108370001500B9C4E019E6F86400DA080085DB00EE
:10838000ECFDECFEECFFF0E82806E04FE6F4200000
:10839000B840E004C4400200C4400400E10CE6F42C
:1083A0002200D7001500B9C4E6F42300D700150059
:1083B000B9C4E6F42400D7001500B9C4F68E76904F
:1083C000D7404E00F48F820BD088DA081676F0D4AE
:1083D0005C4DD7404E00F48F830BD088DA081676B8
:1083E000F084008DC4800400F068D4700200E005C1
:1083F00006F51500DC05B9C7F0470841C440020086
:10840000D7404E00F48F840BD084B84008F3A840C6
:108410003DD7D7404E00D2F88C0BDA081676F0D450
:108420005C4DD7404E00D2F88D0BDA081676004D21
:10843000F1C8E6F42B00D7001500B9C4E10CE6F44E
:108440002100D7001500B9C4F04E49803D15D74032
:108450004E00D2F8890BDA081676F0D45C4DD7407E
:108460004E00D2F88A0BDA081676004DF1C8E6F411
:108470002C00D7001500B9C4D4400200F1C8E6F4BE
:108480001300D7001500B9C4F68E0090F68E029046
:108490003AE8E866F2F476903D08E6F41900E00563
:1084A00022F4009032F502909DF3E6F41900E00505
:1084B00022F4009032F50290ED04E014F6F40A90F4
:1084C0000D1AE6F42300D7001500A9C4F68E7690A5
:1084D000E10CD7001500B9C4E6F42200D70015005E
:1084E000B9C4E6F42400D7001500B9C4E6F42100AD
:1084F000D7001500B9C40806FCFFFCFEFCFDDB003C
:10850000E00BE00CE002E01AF68E0A90D7404E0035
:10851000F68E5000F68E0090F68E02903AE8E866ED
:10852000F2F476903D08F048F058BCF522F4009043
:1085300032F502909DF3F048F058BCF522F400901B
:1085400032F50290ED03E014F6F40A90E6F423000D
:10855000D7001500A984D08648622D03E014F6F4F4
:108560000A90F2F30A903D4F48C1CD0D48912D027B
:10857000E0420D09E6F5E703F04A5C14D7404E00EF
:10858000C454500008A1E6F42000D7001500A984C7
:10859000D08148913D010811F68E7690E00B0D19BF
:1085A000F06BF07BBCF706F6150016F71500F042ED
:1085B000F052BCF500461057DC05A984D08566F55D
:1085C000FF00F04A5C14D7404E00C454500008A18C
:1085D00008B1F0512052405BADE3E10CE6F422001B
:1085E000D7001500B9C4E6F42300D7001500B9C4BC
:1085F000E6F42400D7001500B9C4E6F42100D70042
:108600001500B9C408C148302D85F2F40A904841DC
:108610003D0448C1CD02F68E0A90F04A2841D74069
:108620004E00F6F45000DB003AF7F7FFCA00C888A6
:1086300046FAFF003D1046F780003D1346F9FF0063
:108640003D0746F580003D0D2AF2F2806D0A0D0BC4
:108650004AF2F2800D0846F9FF003D0746F580001A
:108660002D02EA00EE88EA00F68848A02D06489020
:108670003D06F057F046F09AF145EA001889409A15
:108680009D0CF015F057F071F014F046F061F01900
:10869000F09AF0A1F124F145F152F019201A2D0BB6
:1086A00046F119009DEA5AF6F80F7C164AF7F60FC4
:1086B0007C1728113DF82AF2F2806D0E0038104622
:1086C00010579AF5078008915AF4F30F7C144AF575
:1086D000F40F7C15EA000289203830463057EA2032
:1086E00026899D07B1409130914091500831184042
:1086F00018508AF5EF7000331044105528918AF510
:1087000005700044105528919AF5FB70EA000E8917
:10871000CA00C888514546FAFF002D0648A03D1200
:1087200046F9FF002D0D0D1346F780003D0946F96F
:10873000FF002D0348902D040D0F46F580002D0CF1
:10874000EA00EE8846F9FF002D0448903D07EA0054
:10875000268946F580003DF4EA00F688009A26F95D
:108760007E001B57F2F80EFE1B46F2F10CFEF2F3F0
:108770000EFE1B47F2F30CFEF2F40EFE1B56F2F552
:108780000CFE02F40EFE105300411058F178F189EE
:10879000F19AF1ABAAF504702891003310441055FA
:1087A000EA000289F0355C134A88F2107C833A882B
:1087B000F53726F37F009D03E004E005DB00F1BA06
:1087C000F1A9F198E10826F31F002D14FD04E6F449
:1087D000FFFFF054DB0046F3F8FF9D0A06F30800A4
:1087E000F189F19A7C850DF77C144AF5F40F7C151C
:1087F00080033DFA9AF20300814018508150DB005B
:108800009AF603F08140185081507C762B352D0B61
:10881000F1C62D06F0344C564C46A1C06C36705350
:1088200007FC9E000D092B342D0D4C43813006F3BF
:108830008E00F1C6F054E0045C76F189F19A7C85F3
:108840007EF57056DB00CA00C88846F9FF003D156A
:1088500046F580002D042F88DB0040AADB0046FA95
:10886000FF003D0646F780003DF62AF2F2807DF5D6
:108870005C7267F480000941DB0046FAFF003D06A8
:1088800046F780003DE87C1291200DF32AF2F28039
:108890006DEFF0B9F019201A9D02A120F0BA49221B
:1088A0008D059AF20100B130F1430DE3B150DA08C1
:1088B0006A86F0955C197C892D05F01B201947F21A
:1088C00015008DD66810DB00F0955C194A88F2100F
:1088D0007C893A88F537E003E10BF0A75C1A4A88F7
:1088E000F2187C8A3A88F737E008E10FCB00E6F40B
:1088F000FFFFF0540D17E004E6F5807F4AF2F50F14
:108900000D119AF304F0084119A09D0108914890B7
:10891000BD0A46F9FF00DDEF66F57F005C794AF29B
:10892000F90F7059DB00E004E0050DFC1B56F2F571
:108930000EFE1B7402F50EFE1B4602F50CFEF2F451
:108940000EFEDB0048703D20F6F50EFEE606000048
:108950007B66F2F10CFEF2F50EFEF6F40EFEF6F179
:108960000CFE7B66F2F60CFEF2F40EFEE007DB0076
:10897000F0152012F6F40EFEF6F10CFE7B22F2F159
:108980000EFE7C11FFF10D132B17F0274C21E0F3A5
:108990002031F0167C116C13702140529DE9F6F4E1
:1089A0000EFEF6F50CFE7B22F2F10EFE7C116C132E
:1089B0001B61F2F30CFEF2F20EFE1B7102F30EFECF
:1089C000204230539D03281100461057F064F07583
:1089D000F041E005DB00E0089AF504F0E038814062
:1089E000185081509AF705F07A8FF800816018705E
:1089F0008170DA0844899AF80310816018708170D8
:108A00009AF80300814018508150DB00ECF5ECF43B
:108A1000DB0006F0F0FFE10E3AE8E866D74003001D
:108A2000F3F8F72FE4800600D7400300F2F5F42FA7
:108A30005C55D7400300F2F4F42F7CB4004566F493
:108A4000FF00E4800E00F4A00600F1CA67FCF0000D
:108A50002D0447FC1000EA30668BF3F2A0903D66CF
:108A6000F4A00E00C024D7404D00E4A49236258F18
:108A7000A090D7400300F3F8172F67F80F00C084C9
:108A8000D7404D00F6F4923ED4400200D45004008A
:108A900066F4FF00D7404D00F6F47437D74003006A
:108AA000F3F8F82FC084D7404D00F6F47637D7405E
:108AB0000300F3F8F92FC084D7404D00F6F478375F
:108AC000D7400300F3F8FA2FC084D7404D00F6F4E6
:108AD0007A37D7400300F3F8FB2FC084D7404D000E
:108AE000F6F47C37D7400300F3F8FC2FC084D7405E
:108AF0004D00F6F47E37D7400300F3F8FD2FC08415
:108B0000D7404D00F6F48037D7400300F3F8FE2F2E
:108B1000C084D7404D00F6F48237E118D7404D00AD
:108B2000F7F8A53EE118F7F8A2900D1D47F20A00EC
:108B30009D1AE10C0D0BC0C4D7404D00F4A4923631
:108B4000F4800E00418A3D01E11E09C141C28DF34E
:108B500049E03D09F4A00E00C024D7404D00E4A434
:108B60009236258FA0903AE8E86606F01000DB0008
:108B700006F0F0FF3AE8E866F04847F80B003D09D8
:108B8000E7F88800B980E005C4900200C4500400F2
:108B90000D0EE7F88C00B980F0495C84E00506F41E
:108BA000F10016F5DA18C4400200C4500400E7F8DA
:108BB0003000E4800600F3F8A690E4800700F3F8A4
:108BC000A790E4800800E108E4800900E4800A003E
:108BD000E4800B00E4800C00E4800D00E4800E00D3
:108BE000F09066F9FF3FF2FA04FEE018DA08586ADE
:108BF000E018DA08406A06F01000DB0006F0F0FF2B
:108C00003AE8E866F04847F80B003D0DE7F88800C1
:108C1000B980F049C08406F40007E005C4400200B2
:108C2000C45004000D1FE7F88C00B980F04947F8E4
:108C300033003D0CC0845C84E00506F4F10016F5B9
:108C4000DB18C4400200C45004000D0CF049C0847D
:108C50005C84E00506F4F10016F5DA18C440020061
:108C6000C4500400F04AE4800600F04BE4800700A2
:108C7000F04CE4800800D4401000E4800900D440A7
:108C80001200E4800A00D4401400E4800B00D440B9
:108C90001600E4800C00D4401800E4800D00E108C8
:108CA000E4800E00F09066F9FF3FF2FA04FEE0184F
:108CB000DA08586AE018DA08406A06F01000DB00AB
:108CC000F06906F0F0FFF048C088E00976F800F19E
:108CD00076F9DA18E7F88400B980C4800200C490FD
:108CE0000400F09066F9FF3FF2FA04FEC0C8DA080B
:108CF000586A06F01000DB007FE67FE67FE67EE63E
:108D00007EE67EE6E7FC9300E004D7001400B9C4D9
:108D1000E17CD7001400B9C4E7FCBB00E024D70015
:108D20001400B9C4E15CE044D7001400B9C4E7FC06
:108D30003800E084D7001400B9C4E14CE0A4D700A7
:108D40001400B9C4E10CE0C4D7001400B9C4E1CCEC
:108D5000E0E4D7001400B9C4DB00E0060861E024B9
:108D6000D7001400A9846984D0842DF8F068E064E9
:108D7000D7001400B9C4DB00C6030300ECF4ECF622
:108D8000ECF7E0A4D7001400A9E469E40D163AE872
:108D9000E866E064D7001400A9C4C0C6F2F42E90BF
:108DA000248F2E905C14D7404E00C4643605E0A496
:108DB000D7001400A984F1E869E449E0EDE8FCF784
:108DC000FCF6FCF4FC03FB887EE6E7FC1500E044BF
:108DD000D7001400B9C446F908003D2948A03D0653
:108DE000E7FC9300E004D7001400B9C448A13D0695
:108DF000E7FC8700E004D7001400B9C448A23D0690
:108E0000E7FC8300E004D7001400B9C448A33D0682
:108E1000E7FC8B00E004D7001400B9C448A43D5C13
:108E2000E7FC8F00E004D7001400B9C40D55489743
:108E30003D2948A03D06E7FC9200E004D70014005D
:108E4000B9C448A13D06E7FC8600E004D700140041
:108E5000B9C448A23D06E7FC8200E004D700140034
:108E6000B9C448A33D06E7FC8B00E004D70014001A
:108E7000B9C448A43D31E7FC8F00E004D7001400DA
:108E8000B9C40D2A48963D2848A03D06E7FC91004C
:108E9000E004D7001400B9C448A13D06E7FC8400F3
:108EA000E004D7001400B9C448A23D06E7FC8100E5
:108EB000E004D7001400B9C448A33D06E7FC8A00CB
:108EC000E004D7001400B9C448A43D06E7FC8E00B6
:108ED000E004D7001400B9C4F068E007E6F400C26B
:108EE000E015DA08D689F065DA080088DA08A48780
:108EF000F054F6F45C9066F500FFF0457C84F6F4DF
:108F00005A90E6F4FF0064F45C90E15CE044D70022
:108F10001400B9C4E7FCDD00E024D7001400B9C494
:108F2000E7FC6F00E084D7001400B9C4E14CE0A472
:108F3000D7001400B9C4F3FC5A90E0C4D700140061
:108F4000B9C4F3FC5C90E0E4D7001400B9C4E7FCBA
:108F50008500E044D7001400B9C4DB003AE8E866B5
:108F6000F058288148503DFADB00E6F4204EF6F434
:108F7000B2904EE30D083AE8E8669AE204404FE208
:108F80004FE3E108DB00F2F5B290048FB290485055
:108F90003DF2E118DB00E6F4204EF6F4B2903EE339
:108FA0000D1B3AE8E8668AE209304FE2E068DA0829
:108FB0005C8F4EE2E068DA085C8F0D0E3EE23FE324
:108FC000DA086A8F49802D02E118DB00E0A8DA0890
:108FD0005C8F3FE2E108DB00F2F5B290048FB290C3
:108FE00048503DDFE118DB00E6A18000E6A0270045
:108FF000E6201800E6211800E6B004003EE34EE348
:109000003AE8E8668AE20630DA08968F49802D024F
:10901000E118DB008AE20640DA08968F49802D02CB
:10902000E118DB00E108DB003FE24FE23FE34FE302
:10903000E058DA085C8F3EE2E0A8DA085C8F4EE286
:10904000DB00F048F7F8B4904F402E40E7F880007E
:10905000F7F8B5903FE3F78E01F83AE8E866E7F8ED
:10906000800063F8B4902D023FE20D013EE2E7F884
:109070004000F7F8B590DA086A8F6FB06FA1DB0097
:10908000F04861883A884033F78E00F84F402F400F
:10909000E7F88000F7F8B5903EE3F78E01F83AE87C
:1090A000E866DA086A8F6FB06FA1DB00C6030300C1
:1090B000ECF4ECF53AE8E8669A4034204FE2258F6C
:1090C00001F8F3FA01F847FA0800ED1C9AE20530BE
:1090D000F3F8B59075F800F80D05E6F4204EF6F4B7
:1090E000B2904FE2C2F4B5907C14F7F8B5904EE21E
:1090F00047FA08003D433FE39A4002303FE20D3E0D
:109100003EE20D3C47FA09003D3947FA09003D3679
:109110004FE24FE24FE26EB06EB17EB06EA14E40B4
:109120004EE20D2C4FE2258F01F8F3FA01F847FAD1
:109130000800ED156E40F3F8B49063F8B5902D017A
:109140006F40C2F4B5907C14F7F8B5904EE247FA40
:1091500008002D034A40E2630D113EE30D0F47FA6C
:1091600009003D0C4AE2403547FA09003D074FE24D
:109170006EB06EB17EB06EA14E404EE2FCF5FCF4D6
:10918000FC03FB88E6F4FEFFD7000500A844F6F4D4
:109190000690E014F6F40C903AE8E866F68E1E901D
:1091A000F68E1A90F68E2E90F68E1C905FE63AE8B8
:1091B000E866F68E0890F68E0A90F68E1290F68E7D
:1091C0002C90F68E3090F68E3290E0A4F6F4049057
:1091D000E014F6F41690F68E2490F68E3490F6F4A1
:1091E00036903AE8E866F68E2A90F68E3E90F68E35
:1091F0004090F68E4290F68E4490F68E4690F68E13
:109200004890F68E4A90F68E4C90F68E2690F68E0A
:109210002890F68E1090F68E20903AE8E866E009E5
:10922000E6F84200DA08E479E009E6F84400DA08F2
:10923000E479F68E0890E148F7F88A905EEA0EE04D
:109240001EE04EE05EE06FE07FE0DA0872646EE6FA
:10925000E018DA0874766FE63AE8E8663FE84EE828
:109260005EE8F68E0C90DB00C6030300ECF4F2F42B
:109270003A9028412D0A08413D0E248F3A90D18022
:10928000F2E03C90F2A452900D06E6CB0000248F51
:109290003A90E6A41600BF88FCF4FC03FB88F68E27
:1092A000AE90F68EB090E006E0873AE8E866DC071C
:1092B000A986C085E6F4FF002045E00504F4AE90E1
:1092C00014F5B09008611870F046F05726F4FFFFCF
:1092D00036F50800FDEADB00ECFDECFEF0EAF0D824
:1092E00006F0F0FF0EE8F04949813D04E7F88400FC
:1092F000B9800D03E7F88000B980C4B00200C4C093
:10930000040046FD21003D09D4A01200D4901000B5
:10931000E6F85D44DA087E640D2346FD7D003D09D4
:10932000D4A01200D4901000E6F84734DA087E6426
:109330000D1746FDFA003D09D4A01200D49010008C
:10934000E6F8013EDA087E640D0B46FDF4013D08A7
:10935000D4A01200D4901000E6F8003EDA087E6433
:10936000F09066F9FF3FF2FA04FEF04EC088DA088A
:10937000586A06F01000FCFEFCFDDB00ECFDECFE84
:10938000ECFFF0DAF0E8F0F906F0F0FFF09066F9A3
:10939000FF3FF2FA04FEF04DC088DA086268DC4F45
:1093A000A98EE4800600DC4FF48E0100E480070003
:1093B000DC4FF48E0200E4800800DC4FF48E0300E2
:1093C000E4800900DC4FF48E0400E4800A00DC4FE6
:1093D000F48E0500E4800B00DC4FF48E0600E48080
:1093E0000C00DC4FF48E0700E4800D00E108E480FF
:1093F0000E00F09066F9FF3FF2FA04FEF04DC088CF
:10940000DA08586AF04DC088DA08406A06F01000A1
:10941000FCFFFCFEFCFDDB00DA084C00DA081C0057
:10942000DA081295DA082497DA08BC00DA085498AA
:10943000DA08B697DA08F897DA087098DA08D69654
:10944000DA087097DA08F88CDA08E88FE6F480001A
:10945000F6F41CF0E004F6F4DCF1F6F4D0F1F6F4E6
:10946000D4F1E6F97654E6FA0800E6F8013EDA08A7
:109470007E64BF88DB00E6B68000E65A0F00E1F8A4
:10948000F7F87B90E6D81180E6B773006FB74FD836
:10949000DA08189476A840403FE84EE85FE8DA081A
:1094A0008491DA086631FEE2F68E0E901F40E016D7
:1094B000E10AD7404E00E4A6820B86F62502FDF9AC
:1094C000E6F80400E6F92000DA08A4760E40F78EEC
:1094D0007C90F78E7D908A400410E6E30000FA004D
:1094E0000000F2F4089046F450C38D02F68E089006
:1094F0003AE8E8663AE8E866F2F4249028463DEB5C
:10950000D7404E00F78E820BF68E2490DA0808962C
:109510000DE2D180E6E50000E6E00000D180E6E162
:109520000000E6E1FF00E6E20000D180E6E3000093
:10953000E6E31280E6E60000D180E6E70000E6E719
:10954000E000E6E80000D180E6E90000E6E9FF007F
:10955000E6EA0000D180E6EB0000E6EBEF00DB007E
:10956000ECFDF0D8F04849813D0BE019E6F84200E7
:10957000DA08727AE029E6F84200DA08947A0D1CDB
:10958000F04D49823D0BE019E6F84200DA08947A82
:10959000E029E6F84200DA08727A0D0EF04D4983B0
:1095A0003D06E039E6F84200DA08727A0D05E03946
:1095B000E6F84200DA08947AFCFDDB00F0482981E5
:1095C0002D0D29828D102D1429812D1809843D1B04
:1095D0005EEA0EE01EE04EE05EE0DB000FE01EE023
:1095E0004EE05EE0DB000EE01FE04EE05EE0DB0000
:1095F0005EEA0EE01EE04FE05FE0DB005FEA0EE0B7
:109600001EE04EE05EE0DB001E40D7404E00F3F867
:10961000830B07F8CFFF47F809009D5CC0845C24EA
:1096200006F426969C04EA004A96EA005496EA005C
:109630005E96EA006896EA007296EA00AC96EA0046
:10964000B696EA00C096EA00CA96D7404E00F3F8F4
:10965000840B0D40D7404E00F3F8840B0D3BD740F0
:109660004E00F3F8840B0D36D7404E00F3F8840B10
:109670000D31D7404E00F3F8840B07F8CE002D0CC7
:1096800029812D0F09833D261F40E6F80C00E6F9DD
:109690002000DA08A476DB001E40E008DA08BE04E9
:1096A000DB001E40E018DA08BE04DB00D7404E00A5
:1096B000F3F8840B0D0FD7404E00F3F8840B0D0A1E
:1096C000D7404E00F3F8840B0D05D7404E00F3F859
:1096D000840B0D00DB00D180E6E0AA0A66E1FFF80A
:1096E000E6C46B00E6C56700E6C67700E6C765001E
:1096F000E6C96600DB00ECF4E6C60000E014F6F410
:109700001290FCF4FB88B748B7B7FB88ECF4E01480
:10971000F6F47690FCF4FB88ECF4E014F6F4729026
:10972000FCF4FB88E6D81180E65A0F00E6B7730018
:1097300076E2000476E3000466E3FFF7D1807FCE93
:109740007FB6FFD8DB00D1807ECEF6F8B0FEDB001E
:109750007EB7F2F4B2FEDB00ECFF0EFF9AB60270A9
:109760000FFF7EB64AFFF400FCFFDB004FD8DB00A2
:10977000FED9D180E65A630066E2FFDF76E300207F
:10978000E6D93FC076E2002066E3FFFE76E2000203
:1097900076E30002E6BA72007FB9DB00ECF4E01475
:1097A000F6F47490FCF4FB887EB9F6F8B0F0DB00B8
:1097B000F2F4B2F0DB00E6A80000E628579EE629A6
:1097C00019F6E62A579EE62B19F6E6CE5300E6CFA9
:1097D0005700E6C46B00E6C56700E6C67B00E6639B
:1097E000000076A84000DB00248F0890FB88248FBF
:1097F0000090348F0290FB88E6F40004F6F420FF1A
:10980000D1B0E62880FFE62A80FFE6290040E62B5B
:109810000040D190E6BD6C00E6BE5200DB00C603FE
:1098200003003AE8E855FC03FB88B748B7B70DFFDB
:10983000C60303003FE84FE85EE80DFFC6030300E0
:109840003FE84FE85EE80DFFC60303003FE84FE83E
:109850005EE80DFFE6CC6F00E6D08000DB00F2F49E
:10986000A0FEDB00ECF4E014F6F41490FCF4FB88AA
:10987000E6250000E6A40000E6240000E6B45F0050
:10988000E6A30800E6230000DB00FB88A55AA5A597
:109890000A863F001A860212D180E612030C1A894A
:1098A00000FF0A890404E60C0610E68A8004E60D2F
:1098B0000014E68B0004E60E0820E68CAE04E60FEA
:1098C0000015E68D6E04E60A0CFAE6000000E601DB
:1098D0002000E6024D00E60800FCB54AB5B5E6F00A
:1098E0000090FA08769400000000000000000000DC
:02000002F0000C
:10000000DB00DB000000000000000000000000003A
:00000001FF
